:0200000270008C
:1030000000000120793307006133070063330700B4
:1030100065330700673307006933070000000000CD
:10302000000000000000000000000000695F0700D1
:103030006D330700000000006F3307007133070095
:1030400073330700733307007333070073330700CC
:1030500073330700733307007333070073330700BC
:1030600073330700733307007333070073330700AC
:10307000733307007333070073330700733307009C
:10308000A180070073330700733307007333070011
:10309000733307007333070099AB070073330700DE
:1030A000733307007333070073330700733307006C
:1030B00073330700733307000000000000000000B6
:1030C000733307007333070073330700733307004C
:1030D000197A0700733307007333070000000000FC
:1030E00000000000000000000000000000000000E0
:1030F00000000000000000000000000000000000D0
:1031000000000000000000000000000000000000BF
:1031100000000000000000000000000000000000AF
:10312000000000000000000000000000000000009F
:10313000000000000000000000000000000000008F
:10314000000000000000000000000000000000007F
:10315000000000000000000000000000000000006F
:10316000000000000000000000000000000000005F
:10317000000000000000000000000000000000004F
:10318000000000000000000000000000000000003F
:10319000000000000000000000000000000000002F
:1031A000000000000000000000000000000000001F
:1031B000000000000000000000000000000000000F
:1031C00000000000000000000000000000000000FF
:1031D00000000000000000000000000000000000EF
:1031E00000000000000000000000000000000000DF
:1031F00000000000000000000000000000000000CF
:10320000364937480A1A02D0072291438D4635497C
:1032100035480A1A06D00722914381F30988022211
:1032200082F3148831483249324A00F045F8324876
:103230003249334A00F040F832483349334A00F00B
:103240003BF833483349344A00F036F833483449C0
:10325000344A00F031F834483449354A00F02CF84B
:1032600034483549354A00F027F8354835490022B9
:1032700000F02DF834483549002200F028F8344891
:103280003449091A082903DB002202600430016076
:10329000314A90471F482049884205D002680430CF
:1032A00003B4904703BCF7E700208646EC460020B5
:1032B00000212A4A9047FEE7884207D0521A05D0DB
:1032C000037801300B700131013AF9D1704788421F
:1032D00002D002700130FAE77047000000000120C0
:1032E00000F80020000001200000012044E5070054
:1032F0000420002058200020D8330700D8330700CE
:103300000EB1070044E5070004200020042000203F
:1033100010B2070010B2070010B2070010B2070089
:1033200010B2070010B2070010B2070010B2070079
:1033300044E5070098E507005820002058200020A9
:1033400058200020E0610020E0610020E0610020C2
:10335000E0610020E0610020A1330700C96207009E
:10336000FEE7FEE7FEE7FEE7FEE7FEE7FEE7FEE735
:10337000FEE7FEE7704700BF1048804710484FF057
:103380000701884385460F4880470F48016841F48C
:1033900070010160BFF34F8FBFF36F8FFFF730BF36
:1033A0000A480B490B4A884207D0521A05D00378C5
:1033B00001300B700131013AF9D1704775330700C4
:1033C000000001200D82070088ED00E0FCB107003D
:0833D000F01F00200420002082
:1033D8007047000007B5044B0093044A402300F0EF
:1033E80032F803B05DF804FBF933070059200020D8
:1033F8002DE9F84389461446B2B10F4B0F4E032509
:10340800002743F00108224609EB0701002004F0D9
:1034180013F80744241A48B933782BB14FF47A408B
:10342800C047013D02D13570BDE8F88301233370F0
:10343800002CE8D1F8E700BF10B2070058200020A0
:10344800704704F02DB8F0B595B01C4616460846EE
:103458000D4601F060FD1A9B0D93CDE90864002428
:103468002346082205A928460A948DF82C400C9476
:1034780001F07AFD079B0293BDF81830ADF80C30C7
:10348800BDF81A30ADF80E309DF814308DF81140A3
:1034980003F00302012A1DD1BDF81440059EC3F3B1
:1034A800C203C4F383148DF81030A20008230EA9B8
:1034B800284601F059FDC6F3952608AB009322462D
:1034C80002AB0EA9304600F027FC284601F027FD84
:1034D80015B0F0BD022AF8D1BDF81640C3F3C203F7
:1034E800A4098DF810300827082C264628BF08267E
:1034F8003B4632460EA9284601F036FDA41B08AB10
:1035080002AA31460EA8374400F06AFC002CEBD121
:10351800DBE7000008B5FFF794FF0421064800F038
:1035280065FB002803DA0549412000F0E7FD044B5C
:1035380001225A7108BD00BFC4B1070024B20700B8
:1035480004200020037813F0040216D003F00303CC
:10355800012B03D0022B09D0012070470A6800888C
:103568000232C0F3831002440A60F5E70B68428810
:10357800023303EB92130B60EEE71046704700002E
:103588002DE9F04F89B00646871C08A80023484C4F
:1035980000F8113D0D46009200F042FD23682B60B3
:1035A800D4E90123DFF810811344226801339B1A00
:1035B800A8F1040BA8F10809BB421AD3009A00230A
:1035C800002A6DD0012262F3010343F0040366F37D
:1035D80089132168A2689DF80F000A4003320F443E
:1035E80044F82230276000F04BFD012009B0BDE807
:1035F800F08F0121404600F06EFE584600F084FE30
:103608000DF1200A484600F07FFE60684AF8100D68
:10361800A5682840033004EB80005146FFF792FF6D
:1036280002460498002AF4D105EA000304EB830358
:10363800811CDB6805930130054004EB850503F028
:103648000303012B0491ED6823D0022B08D01949FC
:1036580001924FF4BF7000F051FD019A154607E042
:10366800BDF816309B0903332D0C01EB930304932B
:10367800484600F04CFE08B1049B6360294640466A
:1036880000F029FED4E901231344226801339B1A70
:1036980092E7BDF81430C3F383132D0C0B44E6E70F
:1036A800022262F3010343F0040366F39F5390E799
:1036B8006C2100207FB20700883100200D4B0E4896
:1036C80040F2FF3241F2180110B59A6000225A50B8
:1036D80041F21401C3E900225A5003F581531A70CC
:1036E80001F0D2FB044610B9044801F053FC20460F
:1036F80010BD00BF6C21002094B10700C4B20700C0
:1037080030B50A4C71B10A4A0A49121BD208002383
:103718009A4201D1002030BD31F82350854202D0B1
:103728000133F5E7034654F83300F4E724B1070002
:1037380094B10700F01F0020094B013903EBC000CA
:10374800032909D8DFE801F00A02040604207047BB
:103758000079704740797047002070470220704711
:1037680024B10700034BD3E90030C31A584258412B
:10377800704700BF6C2100202DE9F04387B0FFF7A8
:10378800F1FF0646002840F00681844D41F21803F7
:10379800E850BFF34F8F6868AC68DFF8188206AF4F
:1037A80047F8100D2040033005EB80003946FFF73D
:1037B800C9FE029B18B1D8F80020002A61D004EA9B
:1037C8000302991C013305EB8202234005EB8303B6
:1037D800D268DB68049302F00303022B0392029180
:1037E80067D1BDF80E306E484FEA9318B8F1500F04
:1037F800C14628BF4FF0500969F38F1309F108013A
:10380800ADF80E3001F058FB0746002800F0AD80F7
:1038180001F081FB03A900230822384601F08EFB42
:10382800029924EA01060136B600B1453AD95FFA91
:1038380089F9A6B3F6B2A9EB0609214003315FFA6C
:1038480089F4B146574E05EB810108234A463846AC
:1038580001F074FB36B109F10803224631463846B7
:1038680001F06CFB029B08F1030803EB9803029339
:1038780041F21803EB58002B4FD141F21003EC58DA
:103888005EE02A689A4204D86A60304607B0BDE80C
:10389800F08304EA0300033005EB800086E7414922
:1038A8003446D2E72140033108234A4605EB81011B
:1038B800D5E7012B59D1BDF80C303948C3F3831132
:1038C800062928BF062161F3891302318900ADF862
:1038D8000C3001F0F1FA0746002846D001F01BFB36
:1038E8000023082203A9384601F028FB0026BDF86A
:1038F8000C20C2F38312B31C96424FEA8303B7D25B
:1039080002994A1C21400331029205EB81010422ED
:10391800384601F013FB0136E9E7384601F0FFFAB3
:10392800FFF720FF80F00100C6B2AEE7E3685B79DD
:1039380023B1236839461B6820469847E3681C680A
:10394800002CF3D1384601F0EAFA06A800F8114D28
:1039580000F066FB41F21803EB580BB9029B6B6051
:103968009DF8070000F08CFBDAE741F21003EC58F1
:1039780054B90D4B0D480E49C01AC008000440F058
:10398800020000F087F8CBE7236820469B68984739
:10399800E3681C68ECE7002677E700BF6C2100208D
:1039A80094B107007821002024B1070024B1070052
:1039B800D0B20700843100202DE9F74F2F4D804603
:1039C8000F46914601A9012218469B46D5F808A042
:1039D800FFF7D6FD00283DD0019C0026A11C5E45BE
:1039E80006EB010240D10021254800F03EFC80F39F
:1039F800100B244B244A4FEA18499B1AB9EBD30FF2
:103A080004D3224940F2A31000F078FB631C03EAB8
:103A18000A0305EB830349EA0B42DA6004EA0A0366
:103A28000333012115F8232068F3C50205F8232084
:103A380035F8232066F3891225F8232055F823202A
:103A480067F39F2245F8232061F301026FF3820296
:103A580005F823200E4B1B781BB1FFF78DFE0028BD
:103A6800FBD103B0BDE8F08F0AEA020205EB82023F
:103A780059F82630D3600136B1E700BF6C21002029
:103A88008831002094B1070024B107007FB20700F5
:103A98008C31002000231A46FFF78EBF13B502AC05
:103AA800012344F8042D2246FFF786FF02B010BD1B
:103AB80007B5CDE9002302236A46FFF77DFF03B06F
:103AC8005DF804FB1FB5CDE90123069B039301AA0A
:103AD8000323FFF771FF05B05DF804FB1FB5CDE9BF
:103AE8000023069B0293079B03936A460423FFF770
:103AF80063FF05B05DF804FB7FB5CDE90123089BA2
:103B08000393099B04930A9B059301AA0523FFF7D6
:103B180053FF07B05DF804FB2DE9F3478046304CAE
:103B2800D01C8A46174601A900228008A568FFF71D
:103B380027FD002840D0DDF80490A66809F10200AE
:103B4800019001362840361AB6000330B74204EB1C
:103B580080003BD83A46514607F027FA0021214811
:103B680000F083FB80F3100009F101032B4004EB04
:103B780083034FEA184242EA0040D86005EA090385
:103B8800033304EB830214F8231068F3C50104F827
:103B9800231034F823106FF38F1124F82310518861
:103BA80067F38F11518014F82320022161F3010279
:103BB8006FF3820204F823200B4B1B781BB1FFF72D
:103BC800DBFD0028FBD102B0BDE8F0873246514644
:103BD80007F0EBF9BA1B0AEB060104F10C00BBE78E
:103BE8006C210020883100208C31002030B541F252
:103BF80010030F49CA580023144644B9C4682371F6
:103C08005AB941F2100548512260184630BDE4689F
:103C180025799D4206D02468EFE7D26811682160B3
:103C28001060F2E701330A2BE6D14FF0FF33ECE7DF
:103C38006C21002038B541F21002094B9C5803F55D
:103C48008152012313701D4604B938BDE3685D71C4
:103C5800236820465B689847E3681C68F4E700BF60
:103C68006C210020037A052B10B50C460FD0437A3F
:103C780023B1084A0849204600F0F4FB07492046CA
:103C880000F0F0FB2046BDE8104000F0D9BB002A48
:103C9800F8D0F3E71BB307004CBD07003DB307009E
:103CA800C38873B504460D4633B1144A00921449CB
:103CB800144A284600F0D6FB217A05291CD0637ADD
:103CC8004BB1A088FFF738FD0F4B104953F820205F
:103CD800284600F0C7FB227A0D4BA08853F82260D3
:103CE8000021FFF70DFD0B4903463246284602B076
:103CF800BDE8704000F0B6BB02B070BD1BB3070052
:103D080028B3070020B30700E8B207004CBD07003E
:103D18004CB3070040B307002DE9F04385B01F46B8
:103D28000C9D002306460C46904695F80C902B7384
:103D380029463846FFF7B4FFB8F1060F09D8DFE87F
:103D480008F00412181F283340003146284600F0B6
:103D580089FB002229463846FFF784FF85F80C9036
:103D680005B0BDE8F08322683146284600F07AFBAA
:103D7800EFE7D4E900233146284600F073FBE8E773
:103D8800A36800933146D4E90023284600F06AFB73
:103D9800DFE7E3680193A36800933146D4E9002381
:103DA800284600F05FFBD4E723690293E368019398
:103DB800A36800933146D4E90023284600F052FB5B
:103DC800C7E76369039323690293E3680193A368D0
:103DD80000933146D4E90023284600F043FBB8E7B6
:103DE80008292DE9F84F80460E4617461C4636D856
:103DF800002593F80C901D7319461046FFF750FFE5
:103E0800DFF87CA0DFF87CB0AE422AD918F805208C
:103E18005946204600F026FB0135082DF4D11649F5
:103E2800DFF864B0204600F01DFB0025AE421DD926
:103E380018F805A0504607F07DF8002814BF524630
:103E48002E225946204600F00DFB0135082DEDD1F4
:103E5800012221463846FFF705FF84F80C90BDE89B
:103E6800F88F5146204600F0FDFAD5E70349204671
:103E780000F0F8FAE9E700BF16B3070014B307002B
:103E880012B307000CB3070018B3070012F00303BE
:103E980010B511D1094C22604C1CE400A4B2224494
:103EA800074C2260074A1370074A1370074A1080AC
:103EB800074A1846118010BD0720FCE73032002061
:103EC8002C320020283200203832002034320020E2
:103ED800363200202DE9F3472B4D2B888B420646BE
:103EE8000C4617464BD302A84FF0000800F8018D86
:103EF80000F096F8254B264A18781178CBB2254958
:103F080009888B4238BF0133C0B238BF5FFA83F8E3
:103F180040452ED092F800801378DBB2994286BFD4
:103F28000133DBB2002313709DF8070000F0A8F8F6
:103F38004FF6FF73984524D0DFF860A0DAF8003018
:103F48004FEAC80903EB090243F83870A6B19CB1DF
:103F5800114B28881B68224608FB0030314607F0C1
:103F680024F8DAF800304B4400209C8002B0BDE809
:103F7800F0874FF6FF78D7E700209080F6E7092012
:103F8800F4E70420F2E700BF343200203832002082
:103F980028320020363200202C3200203032002017
:103FA800F8B5124C124D264622782B789A4200D149
:103FB800F8BD23780F48104A078812680F48DBB20B
:103FC80019B202EBC10C006852F83120BCF8041099
:103FD80003FB070090470A4A23781288DBB29A420B
:103FE80086BF0133DBB200233370DDE738320020AF
:103FF8002832002034320020303200202C320020B9
:1040080036320020EFF30583C3F308032BB9EFF32F
:104018001480C04300F00100704701207047000081
:1040280070B50446FFF7EEFF012803D0104943207E
:1040380000F064F8EFF3108672B60E4A9068012318
:1040480098B993600C4B0D4DD3F88010294011603E
:10405800C3F88050D3F8841051604FF0FF32C3F892
:104068008420207006B962B670BD2370FAE700BFDD
:10407800B1B307003C32002000E100E0FC06FFBDC0
:1040880010B50446FFF7BEFF012803D009495120A7
:1040980000F034F8084B9A685AB154B9EFF310811C
:1040A80072B6064A18681060586850609C6001B97A
:1040B80062B610BDB1B307003C32002000E100E059
:1040C80030B53AB11368DB430B4C0144884204D144
:1040D800D84330BD4FF0FF33F6E710F8012B5340BB
:1040E800082213F0010F14BF25460025013A85EA7E
:1040F8005303F6D1EAE700BF2083B8ED07B5ADF862
:10410800000001916A46002144F2020002F0AEF874
:1041180003B05DF804FB10B561B1B2FBF3F403FB27
:104128001424A4B244B9C0E9001484608281C38114
:10413800204610BD0E20FCE70920FAE782B050E8BF
:10414800022FC188B2EB324F4FF0000317BF92B273
:1041580041EA014142EA014104E04268B2EB324FD0
:1041680008BF012340E80212002AE8D18DF8073081
:104178009DF80730002B0CBF1120002002B07047BB
:1041880037B550E8013F9DB2C48925448489A542CA
:1041980028BF2D1B0489A54202BFBFF32F8F002221
:1041A80007E0C5EA030540E80154002CE9D14FF0C7
:1041B80001028DF803200193019B9DF803200B60F9
:1041C80002F0FF0322B10B880068184403B030BD29
:1041D8001846FBE70A884B889A4209D150E8012F14
:1041E800C2EA024240E80123002BF7D101207047C0
:1041F8000020704737B550E8023F1FFAA3F5C4887E
:10420800A54202BFBFF32F8F00220DE0C4892544C9
:104218008489A54228BF2D1BC3EA054540E80254FE
:10422800002CE8D14FF001028DF803200193019B87
:104238009DF803200B6002F0FF0322B14B88006851
:10424800184403B030BD1846FBE70A884B889A42E9
:1042580009D150E8022FC2EA224240E80223002B8B
:10426800F7D1012070470020704750E8002F0B4617
:1042780040E8003C9CF0000FF7D11046704750E82A
:10428800002F42EA010340E8003C9CF0000FF6D101
:104298001046704750E8003F43EA010240E8002C0E
:1042A8009CF0000FF6D11046704750E8002F02EA44
:1042B800010340E8003C9CF0000FF6D1104670471F
:1042C80050E8003F03EA010240E8002C9CF0000F90
:1042D800F6D11046704750E8003F03EB010240E872
:1042E800002C9CF0000FF6D11046704750E8003FB4
:1042F800A3EB010240E8002C9CF0000FF6D1104619
:1043080070470121FFF7BBBF0121FFF7C3BF0021A1
:10431800FFF7CBBF0021FFF7D3BF000010B504465D
:10432800002834D003681BB91A49FF20FFF7E6FEBE
:10433800636823B917494FF48070FFF7DFFEA3685D
:1043480023B9144940F20110FFF7D8FEE36823B9F6
:1043580010494FF48170FFF7D1FE238A23B90D4924
:1043680040F20310FFF7CAFED4E9012321689B1A23
:10437800DBB20A60013BDBB2FF2B226802D10020CE
:10438800107110BD1168481C10600B70F2E70E2008
:10439800F7E700BFFBB3070037B5054620B9134957
:1043A8004FF49270FFF7AAFE02A8002400F8014D0E
:1043B800FFF736FE2A686B68116899420ED9481EC5
:1043C800106011F8014CEB68298A01FB0434AB68D2
:1043D80011791B1ADBB2994238BF13719DF8070097
:1043E800FFF74EFE204603B030BD00BFFBB3070009
:1043F80037B50C46054620B9104940F24710FFF77B
:104408007DFE24B90D494FF4A470FFF777FE02A88A
:10441800002300F8013DFFF703FE2A681368591CC2
:104428001160EA68A41A2A8AB4FBF2F41C709DF899
:104438000700FFF725FE03B030BD00BFFBB3070040
:1044480010B5044618B906493120FFF757FEA2688F
:104458002AB163692168206998470023A36010BDC9
:1044680037B407000EB433B5059D044618B9124990
:104478004220FFF743FE63691BB90F494320FFF74A
:104488003DFE23681BB90C494420FFF737FE6368DB
:104498001BB909494520FFF731FE3DB102AA06AB19
:1044A80042F8043D2946204600F06EF802B0BDE807
:1044B800304003B0704700BF37B40700826830B49B
:1044C8000468551C8560A154D0E901329A4202D390
:1044D80030BCFFF7B5BF30BC704700002DE9F84F7E
:1044E8009946DDE90A431746824688460A46012668
:1044F800BA420FD24E4538BF4E4613F0010B01D1D8
:1045080064B900240125B9F1010F1AD909F1FF395D
:104518007D43F8E7B2FBF7F20136E9E79B070ED5D2
:10452800B9F1000F0CBF30252025A642EAD2013C84
:1045380029465046FFF7C2FF002CF6D1E1E72025B7
:10454800F3E7B8FBF5F39F42E2D9DFF83890B8FB00
:10455800F5F3504619F8031005FB1388FFF7AEFF73
:10456800B5FBF7F5002DF2D1BBF1000F02D00CB16D
:10457800A64201D3BDE8F88F20215046013CFFF741
:104588009DFFF4E769B407002DE9F74F0E46904602
:10459800054620B9AC494FF49F70FFF7AFFD6B6932
:1045A80023B9A9494FF4A070FFF7A8FD2B6823B9D8
:1045B800A54940F24110FFF7A1FD6B6823B9A24954
:1045C8004FF4A170FFF79AFD002E00F03A8116F81B
:1045D800011B002958D0252940F0D180002702E08E
:1045E80047F001071646324612F8013B2D2BF7D04B
:1045F800302B04D02B2B05D147F00407F2E747F006
:104608000207EFE700242A2B06F101021BD1D8F894
:104618000030191D1B68C8F800101C441646337872
:104628002E2B1CD101364FF0000A314611F8012B10
:10463800A2F13000092814D80A2303FB0A23A3F1A6
:10464800300A0E46F1E712F8013CA3F130010929BE
:10465800E5D80A2101FB0434303C1646D3E74FF075
:10466800000A324612F8011B01F0FB0068281646C2
:10467800F8D0692916D054D8582970D00ED82529D1
:104688007DD03378002BA2D12B7B002B00F0D98072
:10469800284603B0BDE8F04FFFF7D2BE632968D0C3
:1046A8006429EED1D8F80020D2F80090111D89EACB
:1046B800E972C8F80010A2EBE9724FF0010B092A61
:1046C80061DCD34538BFD3462CB1B9F1000F01DB0B
:1046D800790700D5013CBA0702D5BAF1000F04D01A
:1046E800FB0702D4002C54D10024B9F1000F58DA8A
:1046F800C9F100092D212846FFF7E0FE07F0030263
:10470800022A05D1BAF1000F02D1002C4DD10024A4
:10471800CDE9004753460A2249462846FFF7DEFE00
:10472800AFE7732954D016D87029AAD1D8F8003029
:104738001A1DC8F80020302128461C68FFF7BEFE65
:1047480078212846FFF7BAFE00220823CDE9003277
:1047580021461022E1E775292FD0782991D1D8F880
:1047680000100A1DC8F80020CDE900475346102262
:104778002CE0D8F800301A1D1978C8F8002028460F
:10478800FFF79CFE7DE70A230BF1010B92FBF3F286
:1047980095E7A345A9D220212846013CFFF78EFEC4
:1047A800A0E77807AAD52B21A5E7A345B0D23021E9
:1047B8002846013CFFF782FEA7E7D8F80010CDE9AC
:1047C80000470A1DC8F8002053460A220968A4E7D2
:1047D800D8F800301A1DC8F80020F907D3F800905F
:1047E80012D54F46A7EB090B17F8011B41B9A34592
:1047F800BFF447AF20212846013CFFF75FFEF6E7EC
:104808002846FFF75BFEEDE7B9F1000F17D04846E1
:1048180006F049FC0746BC4200D954B909F1FF39F2
:1048280019F8011F00293FF42CAF2846FFF746FE70
:10483800F6E720212846013CFFF740FEEBE74F460C
:10484800E9E703B0BDE8F08F79B4070070B50D460D
:104858001646044618B908495520FFF74FFC1DB9FC
:1048680005495620FFF74AFC25602B68314620464B
:10487800BDE87040184700BFB2B407002DE9F04109
:10488800DDF818800E4617461D46044618B9224919
:104898008820FFF733FC1FB91F498920FFF72EFC3A
:1048A80023681BB91C498A20FFF728FC1DB91A493F
:1048B8008B20FFF723FC63685A68B5FBF2F302FB11
:1048C80013531BB114498E20FFF718FCB20703D00D
:1048D80011499120FFF712FCBB0703D00E49922023
:1048E800FFF70CFCE3689E4204D36B1E2269334435
:1048F800934203D908499320FFF700FC2368CDF8B9
:104908001880D3F80CE03A462B4631462046F44648
:10491800BDE8F041604700BFB2B407002DE9F0419F
:104928000D4616461F46044618B919499E20FFF73A
:10493800E5FB23681BB916499F20FFF7DFFB1EB96B
:104948001349A020FFF7DAFB63681B68013B2B4281
:1049580003D00F49A320FFF7D1FBE3689D4207D39B
:1049680063681B686A1E03FB06232269934203D906
:104978000749A820FFF7C2FB2368D3F810E03246A6
:104988003B4629462046F446BDE8F041604700BF53
:10499800B2B407002DE9F04108B10368C3B90E4E5F
:1049A8000E4B14229B1B0024B3FBF2F3374602FB89
:1049B80003F5A54201D1002008E03B5930190BB995
:1049C8001434F6E7DB6998470028F9D0BDE8F08190
:1049D800DB69BDE8F0411847F01F002004200020E3
:1049E800014B43600020704700B507000846704738
:1049F80000207047024B1868003018BF012070472C
:104A08004832002008B50248FFF784FC002008BDA2
:104A18004832002008B510461A4606F0C6FA0020AB
:104A280008BD00002DE9F041804686B013480E46C7
:104A380015461F46FFF765FC044630B1112018E003
:104A480006EB043000F092FC0134A542F8D10B4883
:104A5800FFF760FCD8F8083000246BB102226846E2
:104A68008DF80020CDE90146CDE903450597984723
:104A7800204606B0BDE8F0811846FAE74832002023
:104A88002DE9F041804686B012480F4616461D466D
:104A9800FFF737FC0446D8B9AA083146384600F073
:104AA8007DFC0C48FFF736FCD8F8083073B10122BA
:104AB8008DF800200C9A05926846CDE90147CDE9AA
:104AC80003659847204606B0BDE8F0811846FAE726
:104AD8001120F8E74832002029DF704728DF7047A7
:104AE80070B503689D6886B004460E466DB1142201
:104AF8000021684606F082FAA36805932379019697
:104B08002BB1012B0DD06846A84706B070BD012314
:104B18008DF8003023690293E36803936369049373
:104B2800F1E702238DF80030E3681B030293F5E7F1
:104B38000846704700207047024B187A003018BFAB
:104B48000120704738340020034B187A0122B0FA4C
:104B580080F05A74400970473834002008B5104670
:104B68001A4606F022FA002008BD000008B51422F3
:104B78000021044806F042FA0348FFF7DFFA002054
:104B880008BD00BF383400202834002010B5094C77
:104B9800094B43602046FFF7B4FB48B905F0DEFF38
:104BA8001C2320744FF4EE7204490548FFF7B3FA4A
:104BB800002010BD383400202CB507004C320020EE
:104BC8002834002070B5234D234E2B7A2C463BB950
:104BD80022492348FFF70EFB306008B9686070BDB2
:104BE8000223237233681A7972B1012A22D0184637
:104BF8000321FFF775FF00232372636017491848E4
:104C0800BDE87040FFF721BBD3E90520121A142A2A
:104C180028BF1422D3E903159208012A014438BF9A
:104C280001222844FFF758FF50B11128DFD1012392
:104C38002372D4E7D3E903021044FFF74FFFF3E7E9
:104C4800237C002BCBD10146BDE87040022000F048
:104C580009B800BF38340020503400204C340020FC
:104C68002834002038B5831E012B43D8224C237AE0
:104C7800002B3FD0022B09D103282ED01F4B1B68D5
:104C88000022E2601A793AB1012A20D0637C6BBB1A
:104C9800BDE83840FFF796BFD3E905128D1A142DE9
:104CA80094BF521914329A619142EFD102284FF001
:104CB800000308BF19462372104B18BF0D2118684E
:104CC800FFF70EFF0E490F48FFF7BFFADEE71A6934
:104CD80001321A615B699A42E7E7E3680133082BFE
:104CE80001D8E360D2E70023E360DFE7BDE838409E
:104CF80005F024BF38BD00BF3834002050340020F0
:104D08004C3400202834002000F0FD03012B08D18A
:104D1800044B00225A74421E504250411874FFF747
:104D280051BF70473834002010B5064C201DFFF7DE
:104D3800E8FA28B9637C1BB9BDE81040FFF742BF09
:104D480010BD00BF383400202DE9F34180460D46E0
:104D58000F4801A916461F46FFF712FA0446A8B1E4
:104D68001C22002106F04AF92D0B0123237101A909
:104D7800C4F80080A760E56066610548FFF72AFA75
:104D8800FFF7D2FF002002B0BDE8F0810420FAE767
:104D9800283400202DE9F74381468846104801A9A8
:104DA80017461E46FFF7ECF90446B0B11C22002155
:104DB80006F024F900250A9BA36001A92571C4F80F
:104DC8000090C4E9037866610548FFF703FAFFF726
:104DD800ABFF284603B0BDE8F0830420FAE700BF24
:104DE800283400202DE9F74F99469DF8303001937B
:104DF80088461746054618B92249B620FFF77EF9B6
:104E0800EA8895F805B00BFB02FBABF1040BCB4528
:104E180003D81C49C420FFF771F93E68B5F806A00D
:104E280006EB09025A4509F1040188BFABEB0906F4
:104E3800B1FBFAF43E600AFB141144B9AAEB01076E
:104E4800B74228BF37462EB903B0BDE8F08F2D68AA
:104E5800013CF2E7019A043108EB0403681872B1C7
:104E680001463A461846F61B06F09FF8B2453C4400
:104E78002D6857464FF0000128BF3746E3E73A460A
:104E88001946F0E758B50700FFF748BAF8B546796C
:104E98000146721E0546002393422D6803D3002461
:104EA800A64202D8F8BD0133F6E70F682846FFF797
:104EB8009FFA01343946F3E72DE9F843068ACD1CF9
:104EC8000746FFF769FA043E35440446B5FBF6F594
:104ED800F0B14FF48073EDB28380C680013D076066
:104EE80081464FF00008A84512D23846FFF754FA19
:104EF800064648B163790133637108F10108C9F8BE
:104F0800000007608146EEE72046FFF7BFFF344602
:104F18002046BDE8F88301210430FFF7DCB910B55D
:104F2800012104460430FFF7E1F910F0FF0F04D126
:104F38002046BDE81040FFF7A9BF10BD30B585B0C9
:104F4800144604AA002542F8044D0095FFF74AFFCD
:104F5800039BA34203D00349F620FFF7CFF805B01F
:104F680030BD00BF58B5070030B585B0144604AA57
:104F7800012542F8044D0095FFF734FF039BA34237
:104F880004D003494FF48070FFF7B8F805B030BD7E
:104F980058B50700836800225A609A60C3E9042262
:104FA800DA601A607047000038B50D46044618B933
:104FB80009495020FFF7A2F81DB907495120FFF70A
:104FC8009DF82B686A686360934208BF00232560D8
:104FD80008BF636038BD00BF94B5070010B504462C
:104FE80018B90B496320FFF789F823681BB90849EA
:104FF8006420FFF783F8636843B1226891685268B8
:105008000B449342636004BF0023636010BD00BF7C
:1050180094B507000D4930B5A1F594720225914267
:1050280001D800200EE08B1ADB1093FBF5F302EB9E
:10503800C30452F83330834205D802D204F108027F
:10504800EDE7606830BD2146E9E700BF24B70700F7
:1050580008B5FFF7DFFF024B002808BF184608BD58
:10506800E9B507002DE9F04F0022C9B04B780C785C
:105078001B0443EA0463CC7823438C7843EA042373
:1050880008AC0431A3500432402AEFD1234638AD8E
:10509800996B1E464FEAF14282EA714282EA9122F6
:1050A800716A366853F8044F31440A444FEAB441F0
:1050B80081EAF41181EAD4010A449D42DA63E7D116
:1050C800036D0093436D0193836D0293C36D039346
:1050D800036E0493436E0593836E0693DDE905EC36
:1050E800C36E009CDFF8AC900793DDE90381DDE92E
:1050F80001659B4600274FEAF12383EAB11383EA4F
:10510800716A59F827301A4608AB53F827301A4401
:10511800134653442CEA010201EA0E0A82EA0A0203
:105128001A444FEA743A86EA05035A448AEAB40AEA
:1051380006EA050B234083EA0B038AEAB45A0137CF
:105148009A44402F02EB0803E3465244A8461AD17A
:10515800009F1744019A076522444265029A324427
:105168008265039A2A44C265049A1A44059B02661A
:105178000B444366069B73448366079B6344C3667C
:1051880049B0BDE8F08FF44635468E4626461946A6
:105198001446B0E7E0BA070030B5E0B10F4A10494D
:1051A80000240025C0E91245C0E914120D4C0E4A2E
:1051B8000E4DC0E916420E4AC0E918520D4A8266E1
:1051C80002F17452A2F523020023A2F6924203646C
:1051D800C266184630BD0E20FCE700BF85AE67BB2F
:1051E80067E6096A72F36E3C3AF54FA57F520E5195
:1051F8008C68059BABD9831FF8B50446F0B10AB992
:105208000020F8BDD1B10D468E180027B542F7D061
:10521800236C15F8012BE2540133402B2364F5D19C
:1052280021462046FFF71EFFD4E9120110F500724F
:1052380041F10003C4E912232764E7E70E20E0E701
:105248002DE978480D4616460446002800F084806B
:10525800002900F08180026C8021372A02F10103C5
:1052680081544FF000024DD8382B46D1D4E912238F
:10527800206C0821E1FB002322FA01F1934684F80F
:105288003F2084F83E10110C120E84F83C201A0AB4
:105298009C4684F83B3084F83A201A0C1B0E84F89C
:1052A8003D10C4E912BC214684F8392084F838300E
:1052B8002046FFF7D7FE691E7EB30023E26EDA4070
:1052C80001F8012FA26EDA400A71626EDA400A72A2
:1052D800226EDA400A73E26DDA400A74A26DDA408F
:1052E8000A75626DDA400A76226DDA400833202B9F
:1052F8000A77E3D10020BDE87888E2540133B3E7A8
:10530800E25401333F2BFBD921462046FFF7AAFE82
:105318003822002105F072FEA8E71823226DDA4032
:1053280001F8012F626DDA400A71A26DDA400A7243
:10533800E26DDA400A73226EDA400A74626EDA406D
:105348000A75A26EDA400A76E26EDA40083B13F17B
:10535800080F0A77E2D1CDE70E20CCE7024AD2F84F
:105368000034002BFBD0704700E001400A4908B523
:105378000223C1F80435BFF36F8FBFF34F8FC1F815
:105388000805FFF7EBFF0023C1F80435BFF36F8F63
:10539800BFF34F8F08BD00BF00E001400E4B10B5B2
:1053A8000124C3F80445BFF36F8FBFF34F8F01EBA0
:1053B8008204401AA14208D1074B0022C3F80425F1
:1053C800BFF36F8FBFF34F8F10BD431851F8042BF5
:1053D8001A60FFF7C3FFEDE700E0014043689B68F0
:1053E800184708B5436808305A7900F0DDFE0020F8
:1053F80008BD2DE9F0430D469BB0084699469046F6
:10540800FFF7ECFF6E6874794C4528BF4C46074699
:105418002246414602A800F0ABFE727922990AA8FA
:1054280000F0C2FE00970AAB224602A905F1080067
:1054380001F00CFE002848F2425018BF00201BB0B3
:10544800BDE8F0830023C0E90232C0E900118B787F
:105458001A44026191F903301A4442610878003015
:1054680018BF0120704738B54268117803460029F3
:1054780038D002F10C014160147B2CB9C268016874
:10548800FFF7E0FF204638BD5078117900F030056D
:10549800302D14D1547B04F03004302C0FD1907887
:1054A8001969091A19610021907B08441969014496
:1054B800196192F90F20114459610120E3E700F0C6
:1054C800F004202C08D1507910FB01F1002DEBD10C
:1054D800986801309860E7E700F0C000802808BFAE
:1054E8000421F3E70846CEE770B5456804460E4642
:1054F80063681A78B24204D15B7803F00F03082B73
:1055080007D12046FFF7AFFF6368AB42F0D1002018
:1055180070BD0120FCE743681A44426011B10139AB
:105528009A4201D10120704713F8010B01F8010FCD
:10553800F6E7836810B504460BB9002010BD036870
:10554800012298470028F8D0A368013BA360F5E73B
:105558002DE9F3410F460DF107018046FFF7E9FFFA
:10556800064620B90026304602B0BDE8F0819DF815
:105578000740220613D504F07F0407250DF1070123
:105588004046FFF7D6FF0028ECD09DF8072002F030
:105598007F03AB401C43130605F1070501D43C60AB
:1055A800E1E7232DEAD1DDE770B545686A7802F0B6
:1055B8000F06082E86B003461FD103691C68002613
:1055C8000CB906B070BD236862689D6826732946C9
:1055D8006846FFF737FF6368049304F10C030593EB
:1055E8006B7803F0C003802B08BF231D684608BFF3
:1055F8000493FFF7D9FFA468E2E712F0C0011CD1B9
:1056080002F0300010280AD15A691170072EAC68D0
:10561800186909D10146204600F017F8D1E790062D
:10562800F4D55B691970CCE72A79214614B105F0E5
:10563800BCFCC6E705F0E2FCC3E78029C1D10069DC
:10564800002192060160BCD5EBE77FB50A4601460A
:105658006846FFF7F7FE30B16846FFF7A5FF6846D2
:10566800FFF701FFF7E707B05DF804FB30B5044624
:1056780085B01546A9B90268114B9A4211D0102D70
:1056880006D82A4669462046FFF7F0FF05B030BD28
:10569800102269462046FFF7E9FF0028F6D0103DA2
:1056A800EDE7A368AB4201D20020EFE723682A4662
:1056B800204698470028F7D0A3685D1BA560E5E75A
:1056C8001F550700F7B50E4601A907461546FFF70F
:1056D8003FFFA8B1019A0123D3184FF0000404D268
:1056E800717801F0C001802901D1204608E03179A4
:1056F8009942FAD329463846FFF7B8FF019BEC5484
:1057080003B0F0BD73B50D4601A906461446FFF770
:105718001FFF88B1019AFF2A10D86B7803F0C003E5
:10572800802B0BD02979531C994207D32146304648
:1057380001F8012BFFF79AFF02B070BD0020FBE7CC
:1057480010B5034C82600022C0E90041C26010BD60
:105758001F5507002DE9F04F824685B00D464FF0E2
:1057680000084FF0000900240DF10F015046FFF723
:10577800E0FEF8B19DF80F1001F07F025FFA82FB9E
:105788004FF0000CCDE900BC009AA4F1200CC4F144
:10579800200322FA03F302FA0CF71F431346A3402F
:1057A80048EA03080B0649EA070904F1070404D488
:1057B800C5E9008905B0BDE8F08F462CD4D100209A
:1057C800F8E773B50D4669461446FFF7C3FF68B19D
:1057D8002B79082B0CD1DDE90056C4E90056DDE928
:1057E8000023B34206BFAA420120002002B070BDC8
:1057F800042B05D1DDE90001206005460026EEE70F
:10580800022B03D10098208085B2F7E7012B05D140
:10581800DDE90001207000F0FF05EFE70020E5E773
:1058280037B50D4669461446FFF794FF30B12A791B
:10583800082ADDE9003103D1C4E9003103B030BDE5
:10584800042A18464FEAE37108D123601A460B462A
:105858008B4206BF824201200020EFE7022A04D1D2
:105868001BB223801AB2D317F2E7012A03D15BB225
:1058780023705AB2F7E70020E0E7F7B50C4600219D
:1058880019702170116001A9074615461E46FFF7D9
:105898005FFE30B9BB6813B901233370002003B031
:1058A800F0BD01990029F7D0CB0801F007012B6062
:1058B8002170F4E713B5044605291FD8DFE801F085
:1058C800030F151E1E1C012201A92046FFF7CEFE5C
:1058D80018B19DF90430002BF5DB02B010BD082289
:1058E80000212046FFF7C2FEF7E701A9FFF730FEC7
:1058F8000028F2D0019AF3E70422F1E70020ECE750
:1059080073B50D4601A90446FFF722FE064618B9ED
:105918000026304602B070BD94E80F0085E80F00FD
:1059280001998A42F4D3A960A3685B1AA360F0E7DF
:105938002DE9F04155686B7813F0C00E88B0064623
:105948008C46144604D0BEF1400F68D0002544E0D0
:1059580003F00F025C4903F03003102B51F822705A
:105968001DD006D8002BF1D122692946B847054633
:1059780033E0202B17D0302BE8D1636929781970D0
:10598800072A0AD1636820691A79714605F036FB3F
:10599800636821699868FFF758FE22693CE06369EB
:1059A80001221A70E0E7BCF1020FD4F8148027D165
:1059B800042A25D804A9FFF7A3FF05460028C5D067
:1059C800069B2BB1616898F800304A799A4208D84A
:1059D800059B7360069B002BB8D1284608B0BDE82C
:1059E800F0810879226900FB032204A8B84728B18E
:1059F80098F80030013388F80030E1E70546E7E71A
:105A080098F8003021692A7902FB031269799942D2
:105A18009CD9013388F8003061683046A6E71769D9
:105A28003B6807F1040813B9FFF744FF9FE7022911
:105A380013D104A9FFF764FF002887D03B68616889
:105A4800424604A89847054600283FF47FAF069BC6
:105A5800002BF3D1059B7360BFE701292BD009D335
:105A680005297FF473AF04220DEB0201FFF7FEFD59
:105A7800042525E0002501AB591901350B2D3FF40C
:105A880065AF01223046FFF7F1FD00283FF45EAF15
:105A980001AB2B4413F9013C002BECDB0B4B0493BB
:105AA80001ABCDE905350023079342463B686168A1
:105AB80004A898475BE7082201A9FFF7D7FD082546
:105AC8000028EBD142E700BFECBB07001F550700D9
:105AD8002DE9F04F91B00446002604A8CDE90266EE
:105AE800FFF7B0FCA3683BBBDDE9053404A85D788B
:105AF800FFF7B9FC0028F7D115F0300F03D1059B4B
:105B08001B7803B10134002C00F0A980630900223E
:105B180002A9934240F09C8010AA02EB830304F090
:105B28001F04C4F120044FF0FF3053F8383CE04024
:105B3800C31A584258410DE00DF1030301AA0DF1B3
:105B480002012046FFF799FE38B99DF80330002B73
:105B5800CAD1002011B0BDE8F08F019904A8FFF761
:105B6800C3FC002850D1019BB3427FD3059D059A01
:105B7800537803F00F03082B73D004A8FFF773FCC6
:105B8800059B9D42F3D14FF0FF36019FB7426DD37D
:105B9800089B9DF80290D4F808801D684FF0010A10
:105BA800A368002D5FD098459CD12B68D3F800B02E
:105BB800BBF1000F08D04B463A4629462046D84745
:105BC8000028C6D0AD68EBE7D3F808B09BF80030E2
:105BD8009F42F7D16A6859460AA8FFF733FC6B68F9
:105BE8000E9305F10C030F939BF8013003F0C003EB
:105BF800802B04BF2B1D0E930AAA85F80CA04946DA
:105C08002046FFF795FEDBE7059B5B7813F0300F26
:105C18000FD1069A3F2A0CD8510910AB03EB81012A
:105C280002F01F020123934051F8382C134341F826
:105C3800383CE5689DF802201DB104AB0199204667
:105C4800A84704AA9DF802102046FFF771FE12E04B
:105C580051F8225001357FF47DAF013259E7012018
:105C680078E7167891E798457FF43CAF9DF80210E5
:105C78002046FFF71FFE00287FF434AF69E770B5B0
:105C88000C460646154611462046FFF7DEFC2A4616
:105C980021463046BDE87040FFF71ABFF0B585B021
:105CA8000C468D68694607461646FFF729FE68B117
:105CB800A06858B1637803F03003202B3246294698
:105CC800684605D1FFF7DBFF019B7B6005B0F0BD9F
:105CD800FFF7FEFEF8E72DE977480E466946FFF71D
:105CE80039FD88B1DDE90023002502F001045FEAEF
:105CF800530C4FEA320B54EA050308D06FEA0B0243
:105D08006FEA0C03C6E9002303B0BDE87088C6E952
:105D180000BCF9E737B50D4669461446FFF7DBFFC7
:105D280068B12B79082B0CD1DDE90001C4E9000129
:105D3800DDE900238B4206BF82420120002003B028
:105D480030BD042B03D100982060C117F0E7022B67
:105D580004D1BDF90000208000B2F6E7012B04D180
:105D68009DF90000207040B2EFE70020E7E713B587
:105D780004220C460DEB0201FFF778FC08B1019BE9
:105D8800236002B010BD1146FFF7F1BF13B508221A
:105D98000C466946FFF76AFC18B1DDE90023C4E93F
:105DA800002302B010BD1146FFF7F0BF02494FF4BF
:105DB800E870FEF7A3B900BF42BC0700032810B57E
:105DC800044603D908494120FEF798F9074B1C5DA2
:105DD8001F2C01D9FFF7EAFF01234FF0A042A3408F
:105DE800C2F80C3510BD00BF10BC07003EBC070050
:105DF800032810B5044603D908494720FEF77EF961
:105E0800074B1C5D1F2C01D9FFF7D0FF01234FF072
:105E1800A042A340C2F8083510BD00BF10BC07005F
:105E28003EBC070008B50020FFF7E2FF0120FFF79E
:105E3800DFFF0220FFF7DCFF0320BDE80840FFF783
:105E4800D7BFC20710B504460CD54FF0A0430322B4
:105E5800C3F84427C3F84827C3F84C27C3F850278A
:105E6800FFF7E0FFA3070AD54FF0A0430C22C3F8C1
:105E78003427C3F83827C3F83C27C3F8402710BD98
:105E880038B1054B0360054B4360012303720020C2
:105E980070470E20704700BFCF5E0700A95E07005D
:105EA80069B10B78022B0CD1022804D003280CBF4F
:105EB80011200820704703230B70002070470E2024
:105EC80070470820704710B50C4681B10B78042B39
:105ED80004D8DFE803F00E05030E0E00112010BDF4
:105EE80003F0B2FE0028FAD102232370F7E70E2050
:105EF800F5E70820F3E70000F8B50446806916497D
:105F0800164A10F8025C521A0C230E46B2FBF3F242
:105F18003DB92069534300229A4205D101232360E9
:105F280013E04FF0FF30F5E7B758AF4201EB020E30
:105F380006EB020C0ED1471C08D1DEF80850D4E954
:105F48000223D4E90001A8472060F8BDDCF80470FA
:105F58008742F2D00C32DFE718B1070024B10700FE
:105F68001EF0040F0CBFEFF30880EFF30980FFF772
:105F7800C3BF00BF28B139B10023C1E900301846BA
:105F8800704748F21050704748F21350704730B1CC
:105F9800036848F240508B4208BF0020704748F21F
:105FA8001050704728B148F21150914208BF0020A4
:105FB800704748F21050704770B506460C461D46AB
:105FC800FFF7D8FF50B9B3794AB1AB420AD11146AD
:105FD8002046FFF706FA08B9044B236070BD48F263
:105FE8001050FBE748F21150F8E700BF7052464DD9
:105FF8002DE9F0470C4607460F49204615469846B6
:10600800DDE90869FFF7C3FF98B963685A7949461B
:1060180052003046FFF7C6FF58B945B108964346C7
:106028002A4621463846BDE8F047FFF7E2B948F26C
:106038001050BDE8F08700BF7052464D10B50446B9
:1060480038B149B141600B68984708B9044B2360DF
:1060580010BD48F20150FBE748F21050F8E700BFC6
:106068006E524648F0B448B107680A4EB74209D1A3
:1060780059B16AB14368F0BC5B68184748F20150EF
:10608800F0BC704748F20250FAE748F21050F7E7C0
:106098001046F5E76E524648F0B460B107680C4EFA
:1060A800B7420CD171B143681568DC68A5420CD3BE
:1060B8009B68F0BC184748F20150F0BC704748F2A2
:1060C8000250FAE748F21350F7E748F21450F4E7A1
:1060D8006E5246482DE9F041044617469846DDE9D8
:1060E8000656FFF7ABFF60B9424639462046FFF730
:1060F800B9FF30B9324629462046BDE8F041FFF7DE
:10610800CBBFBDE8F0810000F8B50A4F0A4C0B4D33
:10611800E41B0121E40829700026A64203D10223CA
:106128002B700020F8BD57F8363098470028F9D171
:106138000136F2E710B1070010B10700543400200F
:1061480038B50C46054618B908493320FDF7D6FF7F
:10615800611E29442846884200D938BD03780A7848
:1061680000F8012B01F80139F5E700BF71BC070001
:1061780070B50D461446064618B90A494520FDF77C
:10618800BDFF1DB907494620FDF7B8FF621E32441E
:10619800013DB24200D270BD15F8013F02F8013945
:1061A800F7E700BF71BC070070B5164604460D46F8
:1061B800FFF7DEFF3246A919A019BDE87040FFF7C6
:1061C800D7BF38B50D460446FFF7BAFF2946601910
:1061D800BDE83840FFF7B4BF08B507281BD8DFE88B
:1061E80000F004121A1A1A041A040120FFF729FEF3
:1061F8000020FFF7E3FD0120FFF7E0FD0220BDE8E6
:106208000840FFF7F5BD0120FFF7F2FD0220BDE8C9
:106218000840FFF7D3BD08BD08B5FDF70BFDFDF736
:10622800ABFA0028FBD10D4D642445F001054FF46D
:106238007A40A847013CFAD1094B1B68DB0700D517
:1062480000BEBFF34F8F0749074BCA6802F4E062EC
:106258001343CB60BFF34F8F00BFFDE710BD0700AE
:10626800F0ED00E000ED00E00400FA0507B5074B8B
:10627800074C0092E41AE40824040B460246054938
:1062880044F00100FDF71EFCFFF7C6FF24B107002C
:1062980024B10700B4BC070008B5064A064B0749F5
:1062A8009B1ADB081B04024643F00100FDF7F6FBCE
:1062B800FFF7B2FF24B1070024B10700EBBC0700C9
:1062C8000022104638B54FF4805101F029F90246F2
:1062D80008B1FFF7E1FF1F48C0F5FC2101F020F9E4
:1062E80001460028F5D11C481C4CFDF7E7F9FDF7DD
:1062F80011F91B4B1B49E41AE408240444F0030475
:106308002046FDF7C7FB184A18492046FDF7C6FB8B
:10631800174A18492046FDF7C1FB12492046FDF7E8
:10632800B9FB0420FFF78DFD0220FFF747FD4FF072
:10633800A043114AC3F84027104801F0FDF905466B
:106348000028C6D101F0AEF820460D49FDF7A2FBA2
:10635800284638BD00300700717B070024B10700CC
:1063680024B1070016BD070036BD070045BD07006C
:106378004FBD070048BD07000C000300E16107009E
:1063880065BD07008B1802448B4200D1704713F893
:10639800010D02F8010DF7E7C3F10803DB0070B542
:1063A8000133002403A500BF5B1920C940CAAD19F9
:1063B80020C0184720C940CA754120C020C940CA1A
:1063C800754120C020C940CA754120C020C940CAB3
:1063D800754120C020C940CA754120C020C940CAA3
:1063E800754120C020C940CA754120C0644120467B
:1063F80070BD00BF00000000C3F10803DB0070B5EA
:106408000133002403A500BF5B1920C940CAAD1B96
:1064180020C0184720C940CAB54120C020C940CA79
:10642800B54120C020C940CAB54120C020C940CAD2
:10643800B54120C020C940CAB54120C020C940CAC2
:10644800B54120C020C940CAB54120C06441B4FA52
:1064580084F0400970BD00BF2DE9F04F08B4F8CAB8
:1064680004B451F8042BA3FB028940F8048B4FF0C5
:10647800000AE4FB629A4FF0000BE5FB62AB4FF0B9
:10648800000CE6FB62BC4FF0000EE7FB62CE51F851
:10649800042B4FF00008E3FB628940F8048BE4FB0F
:1064A800629AE5FB62ABE6FB62BCE7FB62CE51F8A1
:1064B800042B4FF00008E3FB628940F8048BE4FBEF
:1064C800629AE5FB62ABE6FB62BCE7FB62CE51F881
:1064D800042B4FF00008E3FB628940F8048BE4FBCF
:1064E800629AE5FB62ABE6FB62BCE7FB62CE51F861
:1064F800042B4FF00008E3FB628940F8048BE4FBAF
:10650800629AE5FB62ABE6FB62BCE7FB62CE40F851
:10651800049B40F804AB40F804BB40F804CB40F8B7
:1065280004EB0CBC052B00F01E810C68A0F11400D4
:10653800A1F11401A2F1140252F804EB4FF0000586
:1065480050F8046BE4FB6E5652F804EB50F8047BE9
:10655800E4FB6E6752F804EB50F8048BE4FB6E78AA
:1065680052F804EB50F8049BE4FB6E8952F804EBF4
:1065780050F804ABE4FB6E9AA0F1140052F8044BF7
:1065880051F804EB4FF0000CE4FB6EC540F804CB67
:1065980051F804EBE4FB6E5640F8045B51F804EB49
:1065A800E4FB6E6740F8046B51F804EBE4FB6E788B
:1065B80040F8047B51F804EBE4FB6E8940F8048B47
:1065C80051F804EBE4FB6E9AA0E80006062B00F0F5
:1065D800CA800C68A0F11800A1F11801A2F11802F4
:1065E80052F804EB4FF0000550F8046BE4FB6E56CC
:1065F80052F804EB50F8047BE4FB6E6752F804EBA6
:1066080050F8048BE4FB6E7852F804EB50F8049BC6
:10661800E4FB6E8952F804EB50F804ABE4FB6E9A85
:1066280052F804EB50F804BBE4FB6EABA0F1180081
:1066380052F8044B51F804EB4FF0000CE4FB6EC524
:1066480040F804CB51F804EBE4FB6E5640F8045BC9
:1066580051F804EBE4FB6E6740F8046B51F804EB67
:10666800E4FB6E7840F8047B51F804EBE4FB6E8998
:1066780040F8048B51F804EBE4FB6E9A40F8049B55
:1066880051F804EBE4FB6EABA0E8000C072B6AD0D2
:1066980008B40C68A0F11C00A1F11C01A2F11C02B5
:1066A80052F804EB4FF0000550F8046BE4FB6E560B
:1066B80052F804EB50F8047BE4FB6E6752F804EBE5
:1066C80050F8048BE4FB6E7852F804EB50F8049B06
:1066D800E4FB6E8952F804EB50F804ABE4FB6E9AC5
:1066E80052F804EB50F804BBE4FB6EAB52F804EB31
:1066F80050F804CBE4FB6EBCA0F11C0052F8044B2C
:1067080051F804EB4FF00003E4FB6E3540F8043B0E
:1067180051F804EBE4FB6E5640F8045B51F804EBC7
:10672800E4FB6E6740F8046B51F804EBE4FB6E7809
:1067380040F8047B51F804EBE4FB6E8940F8048BC5
:1067480051F804EBE4FB6E9A40F8049B51F804EB13
:10675800E4FB6EAB40F804AB51F804EBE4FB6EBC11
:10676800A0E8001808BCBDE8F08F002310B51C464F
:106778005AB2914200DC10BD40F823400133F7E7DC
:1067880010B500231A465CB2A14203DCB2FA82F0CB
:10679800400910BD50F8234001332243F3E74A1162
:1067A800012350F8220001F01F0103FA01F108400B
:1067B8007047013949B2002904DA013149B231B9C7
:1067C8000846704750F82130002BF2D0F5E701F168
:1067D8008043013B50F82330002023B9013900EBF6
:1067E800411108B270475B080130F6E710B5002385
:1067F8005CB2A24200DC10BD51F8234040F82340AF
:106808000133F5E710B5013A52B2002A01DA002047
:1068180010BD13B250F8234051F823309C4203D8DE
:10682800F1D24FF0FF3010BD012010BD00EB810107
:106838000023884200D3704751F8042C43EA5203DE
:1068480041F8043DD307F4E770B59DF910401E46A2
:1068580023460546FFF7A0FD30B9224629463046B3
:10686800FFF7D0FF012807D023463246294628469D
:10687800BDE87040FFF7C0BD70BD70B59DF9104010
:106888001E4623460546FFF7B7FD38B12346324674
:1068980029462846BDE87040FFF77EBD70BD2DE94A
:1068A800F04FB5B004AD9DF9F8401F468046234629
:1068B8002846FFF7D1FD24AB2146384602930395BD
:1068C800FFF777FFC0EB841005B26B4203F01F039C
:1068D8004FF0200695FBF6F676B205F01F0914A8CE
:1068E80058BFC3F100093146FFF73FFFB9F1000F68
:1068F80030B22BDD14AB002203EB8000C9F1200E6F
:106908001346A34217D327B27B00019314AB03EBC2
:10691800870704F1FF3934AB012603EB8909002D01
:1069280055DB34AB0022C6F10100964603EB860A1C
:1069380003EB80002DE057F8236006FA09F10A43BB
:1069480040F8232026FA0EF20133DAE714AB224688
:10695800394603EB8000FFF749FFD4E70FFA81FCC3
:106968005AF8C83C53F82CB034AB03EB810151F80A
:10697800803CABEB0303A3EB0E039B4504D034BF71
:106988004FF0010E4FF0000E50F8C81C41F82C30A3
:106998000132019B51B29942E0DBA6EB0E035E4245
:1069A800214614A85E41FFF741FF34AB03EB840393
:1069B800214653F8802C59F8803C384643EAC27384
:1069C800013D49F8803C2DB2FFF730FFA7E734AB13
:1069D80003EB8606224656F8C81C4046FFF706FF1A
:1069E80035B0BDE8F08F30B51C4691B0054693F937
:1069F80000306846FFF730FDD4F8AC3069462846C9
:106A0800984711B030BD13460A46FFF7ECBF2DE991
:106A1800F04793F9006092B0044689461046314623
:106A280015469846FFF7ACFE002840F09380424692
:106A3800494602A8FFF7E7FF434602AA21460AA8EB
:106A4800FFF7D1FF02A908464246FFF7DCFF43469D
:106A58002A4649464846FFF7C6FF08F1040742465A
:106A680029462846FFF7CFFF3B462A4621462046BF
:106A78000096FFF7E9FE3B462A4629462846009637
:106A8800FFF7E2FE3B462A46214628460096FFF7D6
:106A9800F4FE43462A4621462046FFF7A4FF3B461C
:106AA8002246214628460096FFF7CEFE3B46009632
:106AB8002A4621462046FFF7C7FE2368DB074CD548
:106AC80033463A4621462046FFF766FC3146824661
:106AD8002046FFF7ABFE06F18043013B54F8230044
:106AE80040EACA7044F82300424621462846FFF788
:106AF8008AFF3B460AAA294628460096FFF7BDFEAC
:106B08003B460AAA294628460096FFF7B6FE0AA978
:106B180008463B462A460096FFF7AFFE43460AAAB8
:106B280021462046FFF75FFF02AA3B461046214652
:106B38000096FFF7A2FE324629462046FFF756FE8A
:106B4800324649462846FFF751FE324602A94846D2
:106B5800FFF74CFE12B0BDE8F08731462046FFF73C
:106B680065FEC1E72DE9F04115468AB0044688461E
:106B78002022002102A804F041FA2E1D95F9007088
:106B880003232A46414620460293FFF73CFF33463B
:106B980002AA214620460097FFF76FFE2B46424681
:106BA80021462046FFF71FFF0097334605F1840270
:106BB80021462046FFF748FE0AB0BDE8F0810000F4
:106BC800F0B5082289B00C460646FFF70FFECB6ADF
:106BD80003930B6B04934B6B05938B6B0693CB6BF7
:106BE8000793002708236A46694668460297019773
:106BF8000097FFF7D1FB082305466A463146304621
:106C0800FFF7CAFB236B0393636B0493A36B059392
:106C1800E36B0693054408236A4669466846079766
:106C2800FFF7BAFB082305446A4631463046FFF7AA
:106C3800B3FB236A0093636A0193A36A0293A36B6D
:106C48000693E36B0793054408236A4631463046AA
:106C5800059704970397FFF79FFB636A0093A36A5E
:106C68000193E36AA26B0293636B03930492069306
:106C7800E26B236A0592054407936A460823314666
:106C88003046FFF789FBE36A0093236B0193636B3C
:106C98000293236A0693A36A0793054408236A4666
:106CA80031463046059704970397FFF7A5FB236BFA
:106CB8000093636B0193A36B0293E36B0393636A83
:106CC8000693E36A07932D1A08236A46314630462D
:106CD80005970497FFF790FB636B0093A36B0193F1
:106CE800E36B0293236A0393636A0493A36A05938D
:106CF800236B07932D1A08236A46314630460697B8
:106D0800FFF77AFBA36B0093E36B0193636A03932A
:106D1800A36A0493E36A0593636B07932D1A082308
:106D28006A463146304602970697FFF765FB2D1AEB
:106D38000D4C0FD435B9082231462046FFF762FDC5
:106D480001280FD00823224631463046FFF754FB6E
:106D58002D1AEFE70823224631463046FFF71CFB81
:106D68002D18F7D409B0F0BDB4BD0700F0B515462D
:106D780089B01C4607460E461A4629466846FFF75C
:106D880042FE23466A4639463846FFF72CFE23461C
:106D98002A4669466846FFF726FE23466A46314674
:106DA8003046FFF720FE09B0F0BD2DE9F0438BB067
:106DB8001446129D15F9046B00961F4680468946B5
:106DC8002B460246214602A8FFF757FD02A9129A50
:106DD8000846FFF718FE129B02AA41464046FFF7F5
:106DE80002FE129B02AA21462046FFF7FCFD2B4615
:106DF8004A46394638460096FFF73FFD129A39460B
:106E080002A8FFF700FE02A92B4642460846009654
:106E1800FFF733FD02A92B46224608460096FFF7E6
:106E28002CFD2B464246214620460096FFF725FDBD
:106E3800129B224649464846FFF7D5FD2B4602AA33
:106E4800414620460096FFF718FD129B2246394618
:106E58003846FFF7C8FD2B464A463946384600965D
:106E6800FFF70BFD324602A92046FFF7BFFC0BB027
:106E7800BDE8F0832DE9F047B3F9024088461E4685
:106E880004F11F012023073491FBF3F708234FFA7D
:106E980087F994FBF3F4944228BF14464946054603
:106EA800FFF763FC22464146FFF76CFAB6F9023059
:106EB800E4009C4221D9E41A05EB87010022C4F1C1
:106EC80020078D420FD324364A4629463046FFF71D
:106ED80099FC012811D04B46324629462846BDE880
:106EE800F047FFF789BA51F8040C20FA04F313436A
:106EF80041F8043D00FA07F2E3E7BDE8F08770B512
:106F0800036813F001050646144605D013460A46E1
:106F18000146FFF741FA054621463046FFF786FC51
:106F280045B104F18042013A56F8223043F000435B
:106F380046F8223070BDF0B50F46A1B00646194696
:106F4800384615461C46FFF71BFC28B1214630463B
:106F5800FFF70BFC21B0F0BD224639466846FFF723
:106F680045FC2246294608A8FFF740FC214610A800
:106F7800FFF7FBFB0123214618A81093FFF7F5FB49
:106F8800224608A96846FFF73DFC28B9224610A901
:106F98003046FFF72BFCDDE7009BDA0709D42146D2
:106FA8006846FFF743FC2246294610A8FFF7A7FFCB
:106FB800E6E7089BDB0707D4214608A8FFF736FC5D
:106FC8002246294618A8F1E7002823461CDD08AA0E
:106FD80069466846FFF710FA21466846FFF726FC1F
:106FE800224618A910A8FFF70DFC002805DA10A9F9
:106FF80023462A460846FFF7CFF910A9234618AAC0
:107008000846FFF7F9F9CEE708A96A460846FFF7E8
:10701800F3F9214608A8FFF709FC224610A918A889
:10702800FFF7F0FB002805DA18A923462A46084688
:10703800FFF7B2F918A9234610AA0846FFF7DCF9AA
:10704800BEE7000000487047B0BD07002DE9F04FCB
:10705800EDB01F46DDF8D8810590B8F9026098F9BF
:10706800004020231F3696FBF3F676B206F1FF396F
:1070780024AB002543F829506CAB03EB89034CA8DB
:107088008A469346394698F9012043F8805C43F8CC
:10709800605CFFF777F998F9012054A8B918FFF751
:1070A80071F921464CA8FFF76BFB0746002840F012
:1070B8003981214654A8FFF763FB0290002840F06D
:1070C800338108F1240332464CA918460393FFF78D
:1070D80099FB012840F02A81324654A90398FFF70A
:1070E80091FB0128069040F021811CAD0CAF33467E
:1070F800039A54A92846FFF71EFF029B47F8293038
:107108005A46514638464346FFF7B4FE3946384694
:10711800039B00962A46FFF7C2FB0DF5B879039B3F
:1071280000962A464CA914A8FFF7B9FB4846224600
:107138000599FFF75BFBA30009EB030A0793059B7F
:10714800A100591808F1440B50462246FFF74EFBA0
:107158005946224634A8FFF749FBA3000BEB03016D
:1071680022463CA8FFF742FB08F10403494634AA2B
:10717800284600940493FFF780FB53464A463CA9EF
:1071880034A8CDF80080FFF710FE2346049A29465C
:107198002846FFF7D0FE2A46514648464346FFF7A1
:1071A800E5FD029B08933146059B0A933846CDF8C6
:1071B80024B0CDF82C90FFF7FCFA3146814614A88C
:1071C800FFF7F7FA8145B8BF81461FFA89F909F137
:1071D800FF3B0FFA8BFB59463846FFF7E0FA594652
:1071E800071C14A818BF0127FFF7D9FA002814BFF5
:1071F800022300231F430DF1200A22465AF8277064
:1072080024A83946FFF7F2FA0DF1B00BA300F918DC
:1072180022465846FFF7EAFA21462846FFF7A5FA1C
:10722800A9F10209069B2B600FFA89F90DF1900A62
:10723800B9F1000F23DA2346049A29462846FFF7B6
:107248007AFE43462A4659465046FFF78FFD324696
:1072580051460398FFF7D6FA012805D03346039A1A
:1072680051465046FFF7C8F8013C64B2002C4CDA8E
:10727800029BB3FA83F040096DB0BDE8F08F434636
:107288002A46D8F8A47059465046B84749460CA82B
:10729800FFF785FA4946071C14A818BF0127FFF70E
:1072A8007EFA002814BF02200020384308AB53F8A8
:1072B80020702FB32246394634A8FFF797FA079B68
:1072C8002246F9183CA8FFF791FA43462A463CA9FA
:1072D80034A8FFF74BFD049B009434AA514644A8F8
:1072E800FFF7CBFA5B4652463CA934A8CDF800809C
:1072F800FFF75BFD434644AA29462846FFF773FB80
:1073080009F1FF390FFA89F992E723B26CAA02EB67
:1073180083025AF8233052F8802C5340029A1A43B9
:107328000292A1E72846A7E73846A5E70298A3E70F
:107338000369C1688B429DBF8268D21802F1FF328F
:1073480003F1FF3394BF501A581A70472DE9F041E2
:10735800D0E902670446F61B4068964288461546FF
:10736800384405D903F021FE3D44E560BDE8F081CD
:107378003246AD1B03F019FE2A4608EB0601606889
:1073880003F013FEF1E72DE9F843C5680646894680
:1073980017464FF000083469B3687068A54228BFE3
:1073A800E418013C621B5C1BBC4228BF3C4694426B
:1073B80028BF144649462844224603F0F6FDB36820
:1073C8002544AB4208BF00253F1BA044A144F560FB
:1073D800E1D14046BDE8F88310B5114C114AA261CD
:1073E8000223C4E90433104BE361A2644FF48053D1
:1073F8000E4A2362E264002310220D49A362E01DB5
:107408006362E362A3656365E365226503F029FEB1
:107418000849204603F025FE2023A37110BD00BFB4
:107428005834002060BE0700E0340020D03400202B
:1074380069BE07006DBE0700F8B5184C182300FB9D
:10744800033503FB00402544C46A012C0F46164649
:1074580011D003D3022C1BD000240AE02846FFF7E2
:1074680067FF864205D8324639462846FFF76EFF41
:1074780034462046F8BD2846FFF75AFF8642344670
:1074880028BF0446224639462846FFF75FFFF0E743
:107498002846BDE8F840FFF776BF00BF5834002003
:1074A800FFF79ABF70B5184B184C194D1949E41AD3
:1074B800E408240444F004064FF480523046FCF7F4
:1074C800EDFAD5F8802014493046FCF7E7FA4FF07A
:1074D800FF33C5F88030C5F88031C5F88430C5F869
:1074E800843101F0BBFE20B10C4944F00100FCF7E7
:1074F800D1FAFCF741F90028FBD14FF48050BDE8E0
:10750800704000F039B800BF24B1070024B107006B
:1075180000E100E074BE0700AABE0700D4BE070061
:10752800C1F30B0330B52BBBB0F5FE2F22D8000BEF
:10753800013900EB113101254FF08042814201D21F
:10754800002030BD00F01F03440905FA03F3032CA3
:1075580005D8DFE804F00206090CC2F8003601304D
:10756800ECE7C2F80436FAE7C2F81036F7E7C2F8D3
:107578001436F4E70720E4E730B505462148002231
:1075880089B0C0F5FE21FFF7CBFF024648B11E487F
:107598001E4B1F491B1ADB081B0443F00100FCF7B4
:1075A8007DFAEFF305820023D5E9004183F31488BF
:1075B80083F3108883F3118883F31388C2F30802D6
:1075C8003AB984F308884FF0FF339E46084709B05C
:1075D80030BD4FF0FF35203CCDE90033CDE9023313
:1075E8000493CDE905514FF0807320226946204667
:1075F800079303F0DAFC84F30888AE466FF00603BD
:107608001847E4E70030070024B1070024B1070059
:1076180009BF070041DF7047014B01221A7070470C
:107628000049002008B50948094B0A49C01AC00892
:10763800000440F00400FCF72DFA074B074800222D
:107648001A70BDE8084002F0E7BA00BF24B107008D
:1076580024B1070040BF070000490020D176070089
:10766800C31E10B50446042B09D8DFE803F0030352
:10767800080F0F0007494FF4701000F035FA064B59
:107688001B6833B12046BDE810401847FFF7CAFF12
:10769800F5E710BDA57607000449002008B507489E
:1076A800074B0849C01AC008000440F00300FCF763
:1076B800F1F9BDE80840FFF7B5BF00BF24B10700E6
:1076C80024B1070066BF070008B5FCF7B3FAFCF75A
:1076D80053F80028FBD10B4D642445F001054FF405
:1076E8007A40A847013CFAD1BFF34F8F0649074BB0
:1076F800CA6802F4E0621343CB60BFF34F8F00BF48
:10770800FDE700BF60BF070000ED00E00400FA05D8
:1077180008B50648064B0749C01AC008000440F0DF
:107728000400FCF7B7F9002008BD00BF24B107002A
:1077380024B10700B2C0070070B5544B544C5549EA
:10774800E41AE408240444F0040506462846FCF735
:10775800A1F9514B514A1E604FF0A0430020C3F8D5
:10776800402702F089F9064640B900F07DFB012860
:1077780000F0818004D3022800F08580032070BDCA
:107788004FF08043D3F8000410F4803041D04FF418
:107798008032C3F80024304602F060FB002845D14F
:1077A8003F492846FCF776F94FF4701400F086FC40
:1077B8003C4A20211820FCF769FB08B1FEF76CFD54
:1077C8004FF08043D3F81C2512F0B10F1EBFD3F839
:1077D8001C2502F04E02C3F81C25FFF799FF00286C
:1077E800CCD12046304900F07FF9304800F038FE0F
:1077F8000028C3D12E492846FCF74CF900F0A4FC18
:10780800FCF7CEFBFBF7B8FF0028F7D1FFF702FF24
:10781800F4E7D3F8202512F0A90F1DBFD3F82025CF
:1078280002F05602C3F820250120B5E74FF0A04327
:10783800D3F81035DB0301D41E49B2E74FF080437B
:10784800D3F81C3513F0B10F01D01B49A9E702F09A
:1078580033FA002892D1194D2870194802F0DCF942
:107868002B7823B917494FF4CC70FCF747FCFFF786
:1078780019FE154902E0FFF7D5FE144944F001004E
:10788800FCF708F97AE74FF4A0248FE724B1070042
:1078980024B107007ABF0700044900200C00030048
:1078A80091BF0700E0440020A5760700697607002D
:1078B80025C00700B4BF0700D3BF07000049002058
:1078C8002176070035C0070079C00700F4BF07001C
:1078D800F7B5264B06462648C01AC00800040C46D1
:1078E8003246244940F00400FCF7D8F8B4F1807F10
:1078F80037D321498F20FCF701FC6FF07F431F4FDE
:10790800A34228BF2346D7F80455E41A1D44631E32
:10791800942B96BF963474607460347B25F07F4551
:1079280098BF963D032C03D913497720FCF7E6FB53
:1079380004F5A873124A47F823504FF4F86042F050
:10794800010290470F4BA200134400221A601B68E3
:107958000193019B4FF48033A340C7F8043303B06D
:10796800F0BD952CC9D804499020C4E724B107007C
:1079780024B10700F6C007000CC107000040024010
:10798800F0C00700404102401948027884B0002A3C
:107998002BD14FF08043A021D3F81834DB035EBF0E
:1079A800144B01221A60144A0023136012680392D0
:1079B800039A124A136012680292029A104A1360DC
:1079C80012680192019A0F4A82F824131021C2F812
:1079D800841151600C4A0D49C2F8083501230B6027
:1079E80002211360C2F80413037004B0704700BF8B
:1079F8000C4900200800004000410240404102407C
:107A08004441024000E100E00040024008400240DA
:107A18002B4B2DE9F7431A6842B12A490A6801320B
:107A28000A6000221A601B680093009B2648274BB7
:107A3800DFF8B080264EC01AC0080004A8F5102749
:107A480040F00405A7F5A067336823B3002333602B
:107A5800B4003368019307EB040944444A461D49BE
:107A6800019B2846A4F51024FCF718F8A4F2F44367
:107A780019491A784FF480339340184A2846C2F8B7
:107A880008334A46FCF70AF8A4F2FC43196849B1DE
:107A98004846FFF71DFF124B04369E42D4D103B06F
:107AA800BDE8F083A4F59F63196811B14846FFF754
:107AB8000FFFA4F5A0642368002BECD09847EAE7F1
:107AC800044102400849002024B1070024B10700FE
:107AD80040410240CCC00700DEC007000040024021
:107AE800484102400C200020F8B5114B114E0446C5
:107AF80011483768C01AC00800043A460D4640F0DD
:107B080004000E49FBF7CAFF3A7B4FF480339340D9
:107B18000B4AC2F808334CB13668FFF735FF3560B9
:107B280021463046BDE8F840FFF7D2BEF8BD00BF99
:107B380024B107002C20002024B10700CCC0070086
:107B48000040024070B5074B1C6805460E46A06011
:107B5800FFF71AFF266029462046BDE87040FFF768
:107B6800B7BE00BF30200020034A044B1068D3F88A
:107B7800043503EB006070470849002000400240CC
:107B8800014B01221A7070470D4900202DE9F3417D
:107B9800284FFA6A7E6ABC6CAC2A22D17B6B1C44E3
:107BA800F61A254B254D0096ED1AED082D0445F0E3
:107BB80004082346224A23494046FBF783FFFB6A11
:107BC800AC2B14D0324621461D4803F0B8F9B8B999
:107BD8001D494046FBF75EFF0024204602B0BDE881
:107BE800F081002CDDD102F023F90446D9E73246B2
:107BF800A4F58041124803F0A2F90028E8D0E1E793
:107C08003346224611494046FBF752FFFBF7B4FDC5
:107C18000028FBD100F098FA2046314601F0FEFA20
:107C280004460028D9D00A4945F00100FBF732FF85
:107C3800D3E700BF445D002024B1070024B107004A
:107C4800003007005BC10700BDC1070090C10700F5
:107C5800F4C107002DE9F04F3C4B90463C4A9B1A73
:107C680087B0DB081B040493814243F004030546F4
:107C78000E4603930AD10B460A4603983549FBF78B
:107C880017FF0024204607B0BDE8F08F03D2324921
:107C98004F20FCF733FAC5F30B031BB12E495120D3
:107CA800FCF72CFA731B5FEA133B03D12A495420D3
:107CB800FCF724FA00F002FABBF1080F28BF4FF0D6
:107CC800080B08F6FF794FEA0B334FEA1939059389
:107CD800B8F1000F01D14446D4E7CB4534BFDA46AA
:107CE800CA464FF000025146284634BF059F474612
:107CF80001F04EFA04460028C4D12B4632461749F3
:107D080003980097FBF7DEFEFA1C234622F00302D5
:107D18003146284601F0FEF904460028B2D1104A3F
:107D2800136BA8EB07083D443E441F44176301F05A
:107D380079FFA9EB0A0904460028C9D0049B094920
:107D480043F00100FBF7A6FE9CE700BF24B1070043
:107D580024B107000EC207003CC207008EC207000C
:107D6800445D0020AFC207002DE9F04702F072F829
:107D7800344C354BDFF8ECA03449DAF84850DAF8DF
:107D88003080DAF83460E41AE408240444F0040784
:107D980081463846FBF77EFE42F20403EA5803F1B7
:107DA800A34303F5471303F2D7539A4208D028494F
:107DB80044F00100FBF76EFE03252846BDE8F08776
:107DC800DAF83020B242154405D122493846FBF78B
:107DD80061FE0025F1E7DAB94FF4405338461B78C5
:107DE800142B81BF43F214031A681B4BB2FBF3F246
:107DF80005F500531B78142B81BF42F21403164972
:107E0800EB58B3FBF1F398BF00231449FBF750FE7E
:107E1800A6EB080202F6FF7222F47F62294622F0DE
:107E28000F0209EB0800FFF715FF054628B10C49BA
:107E380044F00100FBF72EFEBFE7BDE8F04701F074
:107E4800F1BE00BF24B1070024B10700B5C4070084
:107E5800DAC407000EC5070040420F0020C507001E
:107E680049C50700445D00202DE9F0475B4B5C4C99
:107E78005C4F5D49E41AE408240444F004084046D1
:107E8800FBF708FEFB6AA52B7AD009D8012B1FD077
:107E980044F003005549FBF7FDFD0020BDE8F087DD
:107EA800AA2B78D0AC2BF3D151494046FBF7F2FD11
:107EB80050494046FBF7EEFDFFF756FF0546002800
:107EC80072D04D4944F00100FBF7E4FD012620E0A3
:107ED8004A494046FBF7DEFD7E6AD7F8489001F034
:107EE80091FF3D6B464900EB050A4046FBF7D2FD82
:107EF800396B49448A4514BF721B00225046FFF76C
:107F0800A9FE054668B13F4944F00100FBF7C2FDF0
:107F18000026FB6A3C492A4644F00100FBF7C8FDED
:107F280012E001F06FFF2A463146FCF7C9F8BA6A39
:107F3800904281461DD135494046FBF7ABFD0123F0
:107F4800C7E90793BE612E463148324D01F04EFF16
:107F5800002331482B7001F065FE2B78074623B9C2
:107F68002E4940F2A310FCF7C9F887BB26BB0120B5
:107F780094E703462A4944F00100FBF799FDE2E73C
:107F880028494046FBF786FDFFF7EEFE0126054629
:107F9800002DD9D0BDE724494046FBF77BFDFFF70C
:107FA800F5FD00260546F3E7FFF7F0FD054608B1A5
:107FB8001E4987E70126C7E7012001F04FFF002887
:107FC800D5D040461A49FBF765FD022066E744F024
:107FD80001001849FBF75EFD03205FE724B10700A5
:107FE80024B10700445D0020E8C20700F4C307007D
:107FF8009DC30700ABC30700C8C3070009C3070038
:1080080013C3070049C507000DC407002EC30700A6
:10801800685D00200D490020897B07003CC20700ED
:1080280043C307008BC3070094C30700DEC30700E0
:108038003FC407009BC407000A4AD2F800347BB14A
:1080480009480023D2F80815D940C90748BF03F5E5
:10805800C07103F1010348BF42F82100072BF1D199
:10806800704700BF000001403546526E08B507480A
:10807800074B0849C01AC008000440F00300FBF78A
:1080880009FDBDE80840FFF7D7BF00BF34B10700BE
:1080980024B10700D3C5070007B5074B00221A60B3
:1080A8001B680193019BFBF7C5FDFBF765FB0028E7
:1080B800FBD103B05DF804FB0001014070B5194E17
:1080C80033784BBB184C1949194B641AE408D3F898
:1080D8000024240444F00304FAB1D3F804551549E4
:1080E8002A462046FBF7DAFC40F616539D42B8BFF5
:1080F8001D46A5F54865FFF79FFF2A460E4920460D
:10810800FBF7CCFC0D492846FFF71CFD0C4B4FF440
:1081180080321A600123337070BD0A492046FBF78C
:10812800B9FCF7E70E49002034B1070024B1070075
:108138000000014062C507007BC507007580070085
:1081480000E100E0ADC50700034BD3F800340BB1E4
:10815800FFF772BF704700BF0000014013681F2B74
:1081680010B5144607D900220830FDF769F808B998
:108178002023236010BD48F21450FBE70830FDF7B8
:108188003BB80830FDF708B8007800F001007047E8
:108198000C4B1B78062B10D10B4B1B681A070CD104
:1081A8000A4B186800F0F003302B08D000F0E0000C
:1081B800A0F1400358425841704700207047012001
:1081C800704700BFE00F00F0E40F00F0E80F00F088
:1081D800094B1B78062B0CD1084B1B681A0708D1D2
:1081E800074B186800F0F000A0F1300358425841DE
:1081F80070470020704700BFE00F00F0E40F00F068
:10820800E80F00F008B5FFF7C3FF28B1774B784AAD
:108218001B68C3F304231360FFF7DAFF10B1754B33
:10822800754A1A60FFF7B4FF28B1744B744A1B688B
:10823800C3F342331360FFF7CBFF20B1714AD36811
:1082480023F08073D360FFF7A3FF40B14FF0804362
:108258000022C3F80C21C3F81021C3F83825FFF712
:10826800B7FF10B1684B03221A60FFF7B1FF40B1A6
:10827800664B05221A6001229A6700229A603F2203
:108288005A60634B1B78062B50D1624B1B68190749
:108298004CD1614B1B6803F0F003502B46D14FF0D3
:1082A80080525E4BD2F80414C3F82015D2F8081493
:1082B800C3F82415D2F80C14C3F82815D2F81014F2
:1082C800C3F82C15D2F81414C3F83015D2F81814C2
:1082D800C3F83415D2F81C14C3F84015D2F820148A
:1082E800C3F84415D2F82414C3F84815D2F8281452
:1082F800C3F84C15D2F82C14C3F85015D2F8301422
:10830800C3F85415D2F83414C3F86015D2F83814E9
:10831800C3F86415D2F83C14C3F86815D2F84014B1
:10832800C3F86C15D2F84424C3F87025FFF730FF62
:1083380028B13B4B3B4A1B6803F04F031360FFF720
:1083480027FF48B14FF08043D3F80024D20744BF39
:108358006FF00102C3F80024334AD2F8883043F49E
:108368007003C2F88830BFF34F8FBFF36F8F4FF0A1
:108378001023D3F80022002A03DBD3F80432002BA1
:108388002FDA2A4B0122C3F80425D3F80024002A47
:10839800FBD04FF010221521C2F80012D3F80024A8
:1083A800002AFBD04FF010231522C3F804221F4BDC
:1083B8001A46D3F800140029FBD00021C3F804158D
:1083C800D2F80034002BFBD0BFF34F8F1649184B5F
:1083D800CA6802F4E0621343CB60BFF34F8F00BF5B
:1083E800FDE7144B144A1A6008BD00BF24030010AF
:1083F8004035014074C007400DF0ADBA440200108A
:108408003C050040F0ED00E0A0050040105600409B
:10841800E00F00F0E40F00F0E80F00F000C00040AB
:1084280058020010E40E004000ED00E000E00140BA
:108438000400FA05342000200090D003062810B567
:10844800044602D1002001F097FC044B1B681BB1C5
:108458002046BDE81040184710BD00BF1049002055
:1084680038B5104B104C1860104B1149E41AE40849
:10847800240444F00300FBF70DFB0020FFF7DEFFA8
:108488000C4801F041FC054620B90A48BDE83840CF
:1084980001F04EBA0246084944F00100FBF7FEFA23
:1084A800284638BD1049002024B1070024B1070030
:1084B80014C707004584070027C707006CDF70470B
:1084C8006DDF704772DF704773DF704774DF704786
:1084D80075DF704776DF70477ADF70477CDF70475B
:1084E8007DDF70477FDF704786DF70478FDF70471B
:1084F80090DF7047A8DF7047AADF7047ADDF70478D
:10850800AEDF7047B0DF7047B1DF7047B5DF704747
:1085180062DF704766DF704713DF70477FB500235F
:10852800CDF80A30ADF80E300A4BADF806109B892D
:10853800ADF8083001238DF80A300DF10603CDE9B6
:108548000430054B02A91888FFF7DAFF07B05DF879
:1085580004FB00BF7E5900203A20002010B5094BCB
:10856800094904460948C01AC0080004224640F0D8
:108578000400FBF793FA21460548BDE81040FBF7D5
:1085880037BF00BF24B107007ECC07003CB107000D
:10859800A8B1070030B518228DB00DEB02000021FC
:1085A80002F02CFD282308932448254B2549C01A9E
:1085B800C0080004012440F004008DF818408DF82C
:1085C8002D40FBF767FA1623ADF806300023CDF8E7
:1085D8000E30CDF81230ADF816301B4B0293022244
:1085E800062109251A7099701A7103215922D97028
:1085F8005A710DF10601FE225819ADF80C505C7045
:108608009A71FFF76DFFB8B9BDF806201D721119F0
:10861800D971BDF80C301A440C4BADF80C2002A9E6
:1086280006AA1846FFF74EFF30B91878FFF74EFF35
:1086380021461878FFF748FF0DB030BD3CB1070060
:1086480024B1070061C70700925900203820002094
:10865800F0B50388212B8DB0044600F06A8132D82A
:10866800122B00F0398107D8102B56D075D8012B62
:1086780000F0AA810DB0F0BD142B00F03782C0F0D5
:1086880001811A2B00F043821F2BF3D1B24BB34D5B
:10869800B349ED1AED082D0445F00400FBF7FAF98B
:1086A800B04B04F108011888FFF712FF04460028B0
:1086B800E0D00246AC4945F00100FBF7EFF920464F
:1086C800FDF7EAFDD6E7502B5CD013D8232B00F03A
:1086D800C780C0F01F81242BCCD19F4B9F48628953
:1086E800A249C01AC0080004E38940F00400FBF75F
:1086F800DFF9BFE7522B00F00A82C0F06B81552BDF
:1087080000F08280562BB5D18379002BB2D1954BDE
:1087180013211888FFF7DEFE9AE08F4B8F4D94499E
:10872800ED1AED082D0445F00400FBF7B3F98D4B65
:10873800A2881A808F4A12681C460AB10120904705
:108748008D492088FFF7C4FE0246002892D08B4945
:1087580045F00100FBF7A2F98CE7824B4FF6FF7258
:108768001A80874B1B685A0704D4FFF713FF08B118
:10877800FDF792FD7F4B1B68002B3FF47BAF022077
:10878800984777E77F4FC288BB889A427FF472AFD9
:108798007D48724DFBF700FE6F4BED1AED082D0476
:1087A800064628B9794945F00200FBF773F961E7F5
:1087B800F422238A76490092024645F00400FBF72A
:1087C80081F9228A04F11201304602F0EEFB1822E8
:1087D80000210DEB020002F011FC08238DF818307F
:1087E8006C4B08936C4B0797CDE9093606A8238A8A
:1087F800ADF82C3001F07CF800283FF43BAF31464F
:108808006148FBF7F5FD35E7C288F62A24D8D31E60
:108818009B0723D0D31F9BB2013B594201F00301B0
:1088280003F0030302F1FF3458BF4B42E31A9CB232
:10883800494B4A485949C01AC0080004234640F029
:108848000400FBF735F9474B21461888FFF75EFE11
:1088580000283FF40FAF33E7F724E9E71446E7E7CA
:108868003D4B3E484E49C01AC008000440F0040081
:10887800FBF710F9002206A9A088CDE90622FFF728
:1088880037FEE5E7344B354C4649364DE41AE408E3
:10889800240444F004042046FBF7FCF80023ADF858
:1088A8001A300223ADF8183006AA04AB42F60521A7
:1088B80028880793FFF722FE08B1FDF7EDFCBDF805
:1088C800102039492046FBF7E9F800231A4685218C
:1088D8002888FFF707FEBBE71F4B204D3349ED1AE9
:1088E800ED082D0445F004052846FBF7D3F8628906
:1088F8002F492846FBF7D2F822892E492846FBF74C
:10890800CDF8A2892C492846FBF7C8F8E2892B49FB
:1089180028461FE7437A827A0F491048401AC00850
:10892800217A00910004264940F00400FBF7CAF8B8
:10893800A0E6094B09482349C01AC008000440F0C2
:108948000400FBF7A7F80CA9002321F8183DA0881C
:10895800FFF7CCFD7CE700BF24B107003CB107005E
:108968001ACB07003A20002049CB070017CA070096
:1089780029C90700B859002076CC070033C9070079
:10898800B45900207E590020A8B1070061C907002A
:1089980080C90700198C070065850700A0C9070072
:1089A800E6C9070055CA07007DCA0700A0CA070024
:1089B800C7CA0700DDCA0700F3CA070005CB0700CE
:1089C8007ECB0700B8CB07005A4B00211888FFF769
:1089D800A1FD3DE78379002B3FF44CAE022B7FF4D9
:1089E80049AE554D0289AB899A427FF443AE837BE9
:1089F800012B7FF43FAE00230121CDE906338DF82A
:108A08001E10018AADF820104A4E418AADF8221096
:108A1800022200F114018DF818200991ADF81230E6
:108A2800ADF8102003AB298A3088059304AAFFF714
:108A380065FD374660B91846FFF7A6FB40B940F216
:108A4800FD1306A93088ADF81C30FFF75BFD11E671
:108A5800002306A93888ADF81C30FFF753FD0146FE
:108A680000287FF407AE18220DEB020002F0C6FAC8
:108A7800237D324A8DF81830022B0795089222D0B0
:108A8800062B0ED0012B0ED12D4801F075F92D4B78
:108A98001A882D4B1A80637D0A93D4F816300B93ED
:108AA80001E0637D0A9306A800F022FF0246002831
:108AB8003FF4E0AD2548264B26491B1ADB081B046A
:108AC80043F0010046E6214B21482349C01AC0085B
:108AD800000440F00400FAF7DDFFA27D637D43EA5D
:108AE8000223184A1380184A1380DCE7174B1848EA
:108AF8001A49C01AC008000440F00400FAF7CAFF77
:108B080000231A461946A088FFF7EEFCA0E60023CA
:108B18001A461946A088FFF7F7FC08B1FDF7BCFB19
:108B28000B480A4B0E49C01AC008000440F0040064
:108B38003BE600BF3A2000207E590020198C070030
:108B480010B10700BC590020BE59002024B107000D
:108B58003CB10700F3CB0700E1CB070027CC0700A7
:108B68004DCC070070B5204E346814F0010432D0A3
:108B78001E4B984236D01E4B1E4D1F4C1F49ED1AF6
:108B8800ED082D0445F004052846FAF783FF2288EE
:108B98004FF6FF739A4220D019492846FAF77AFF10
:108BA8003368208843F0040313213360FFF792FCF5
:108BB800044680B9134EC82446F001064FF47A40A3
:108BC800B047013CFAD101F089FF044618B90E49B3
:108BD8002846FAF75FFF204670BD0C4B1878FFF760
:108BE80075FCF0E70024F6E7B459002010B107003F
:108BF80024B107003CB107003A200020E0C7070075
:108C0800FDC7070070CC07000CC8070038200020FB
:108C180030B50D4687B0044620B9464940F28F105A
:108C2800FBF76CFA25B943494FF4C870FBF766FAAD
:108C38001122002101A802F0E1F92378082B0BD1B9
:108C48003D4A3E4913880988013B9BB2138031B3E2
:108C58002BBB032311802370637822788DF80520BD
:108C68006021012B8DF804108DF8063019D0344995
:108C78003448401AC0080004334940F00200FAF7AB
:108C880017FF63780B2B52D100F0BEFA8DF807005E
:108C9800002000F0B3FA042101A8FFF73FFC07B059
:108CA80030BD062A1DD0082A01D0032A3FD1D4E9B5
:108CB8000123110A8DF807208DF80810110C120EE7
:108CC8008DF80A201A0A8DF80B308DF80C201A0C32
:108CD8001B0E8DF809108DF80D208DF80E300B2124
:108CE800DAE7E1688DF80710D4E90123080A8DF85E
:108CF8000800080C090E8DF80A10110A8DF80B20CF
:108D08008DF80C10110C120E8DF80E201A0A8DF821
:108D18000F308DF810201A0C1B0E8DF80D108DF8E1
:108D280009008DF811208DF812300F21B4E70321C6
:108D3800B2E700BF70C70700BE590020BC59002029
:108D480024B107003CB10700B9C707002DE9F0437B
:108D5800804695B020B9504940F25240FBF7CEF911
:108D68004E4B4FF6FF7214A91A804FF65963012033
:108D780021F8483D42468DF80A00FFF7BBFB044640
:108D8800002840F08580464B04AA03F110061546DA
:108D980018685968144603C40833B3422246F7D109
:108DA80008F102012846FFF7B3FB044600286FD1FB
:108DB80001461C220DA802F021F99DF83430ADF8C7
:108DC800044043F004038DF834300223ADF80C302E
:108DD80098F802308DF80E304FF00109C4F30723DC
:108DE80069F3030369F307138DF80530E3B243EA27
:108DF800090369F342038DF80630F423CDE90A44E8
:108E080001ADADF82C3003AE08F1040308AA0DA992
:108E1800B8F800000C94CDE90865FFF76DFB27460C
:108E28000446A8BB01461C220DA802F0E7F89DF8ED
:108E38003430ADF8044043F018038DF8343098F816
:108E480002308DF80E30C4F3072369F3030369F386
:108E580007138DF80530FBB243EA090369F34203AF
:108E6800DBB243F010038DF806301723CDE90A442E
:108E780008AAADF82C300DA908F10C03B8F80000C9
:108E88000C94ADF80C90CDE90865FFF735FB044666
:108E9800204615B0BDE8F08370C707003A200020CF
:108EA80051C70700F0B5524E336813F0010485B07E
:108EB800074640F09B804F4B4F4D5049ED1AED0847
:108EC8002D0445F004052846FAF7E4FD4C4B4D48BF
:108ED8001F60FBF723FA029400F0B1F9044600285A
:108EE80073D1494A49492846FAF7D8FD4648FFF759
:108EF80013FB0446002868D145492846FAF7CAFDFD
:108F080001F0B0FD044600285FD102A801F076FE0A
:108F18000446002859D13F492846FAF7BBFD02A963
:108F2800012001F075FE044600284ED13A49284632
:108F3800FAF7B0FD02A801F03BFF0446002844D12F
:108F480000F0AAFE002843D0344800F099FE3368A8
:108F580043F002033360112302A88DF80430FFF7B1
:108F6800AFFA044688BB9DF8093002A801338DF892
:108F78000930FFF7A3FA044638BB33689B072CD5A2
:108F8800264C2749A3692846221DFAF791FDA069B6
:108F9800211D82B201A8FFF7A1FA0446A8B9214809
:108FA800FFF79AFA044680B91F48FFF7CFFE044638
:108FB80058B9FFF7EFFA044638B933681B4943F04C
:108FC800010328463360FAF765FD204605B0F0BD79
:108FD80017492846FAF75EFDBDE716492846FAF70D
:108FE80059FD154802F05FF81349D2E70024ECE771
:108FF800B459002024B107003CB107002DC8070070
:10900800B8590020A8B10700003007004CC8070075
:109018006CC8070081C8070098C8070014490020D9
:10902800CAC8070076CC07007E5900200AC9070085
:10903800B0C80700EBC8070025C8070030B51A49B3
:109048000B6885B004460BB1013B0B601748184A02
:1090580063682578801AC008000440F004008BB9C2
:109068000B68144A14490093012D18BF0A46A368D7
:109078001249FAF727FD63699BB1E06805B0BDE8BE
:10908800304018470A68029222690192A268009249
:109098000949084A012D18BF0A460949FAF72CFD63
:1090A800E9E705B030BD00BFC059002044B1070052
:1090B80024B107009CCC0700A2CC0700A8CC07006D
:1090C800CECC070008B50C4A0C4B9B1ADB081B04D6
:1090D80043F0040350B10A491846FAF7DBFC094982
:1090E80009480022BDE80840FBF7B0BB074918460D
:1090F800FAF7D0FC0649F3E724B1070044B10700AA
:1091080074CD070038B50700F01F00209ACD07007E
:109118000CB507002DE9F7439846174C174BDFF8B5
:109128006C90E41AE408D9F8003024040546CDE927
:1091380000230E460B4617461149024644F0040028
:10914800FAF7CCFC2946CDF800803B4632460D485C
:10915800FBF794FB054640B9D9F800300133C9F84C
:109168000030284603B0BDE8F0830246064944F0C3
:109178000200FAF793FCF4E744B1070024B10700B2
:10918800C2CD0700F01F002005CE0700C0590020FF
:109198002DE9F341134B144C144EE41AE4083368D8
:1091A8000093240405460B460F4690461049024694
:1091B80044F00400FAF786FC294643463A460D482F
:1091C800FBF7ACFB054630B93368013333602846FA
:1091D80002B0BDE8F0810246074944F00200FAF700
:1091E8005DFCF4E724B1070044B10700C059002032
:1091F8000ACD0700F01F002047CD0700014B18706B
:109208000B207047C4590020024B002218781A70AE
:10921800704700BFC459002018DF704730B585B0CB
:10922800054610220C466846002101F0E7FEA40816
:10923800684601950294FFF7EFFF05B030BD1FB5F2
:10924800002304A8CDE901330393022340F8103D1D
:10925800FFF7E2FF05B05DF804FB000010B50B4B0B
:109268000B4C0C49E41AE408240444F00404204696
:10927800FAF710FC4FF000534FF4805220461A6062
:109288000549FAF707FC002010BD00BF24B107000C
:1092980024B1070046CE070040CE0700084B094816
:1092A8000949C01A10B5C008000440F00400FAF7D4
:1092B800F1FB064B06201B68BDE81040184700BFAD
:1092C80024B107004CB107000ED40700D059002084
:1092D8000A2803D90B38C0B2FFF790BF70470000C7
:1092E80070B5054686B00020FBF754FB014690B1E7
:1092F800244A18212846FAF7EDFD024648B12248CB
:10930800224B23491B1ADB081B0443F00100FAF720
:10931800C5FB06B070BD1822684601F06FFE042335
:109328008DF80030194C184B1A4EE41A1A4B1A6D66
:109338003368E40824049A4244F004041AD1174913
:109348002046FAF7A7FB164B3168186801F024F994
:109358008DF80100FFF7BCFFD5E901138DF8010076
:10936800684698470F4800F05DFC9DF801200E49BB
:109378002046CCE701238DF801306846D5E9011372
:109388009847F2E7E992070024B107004CB10700BB
:109398008ED30700C8590020445D0020B7D30700CA
:1093A800CC590020A5920700E6D30700F0B58368E2
:1093B80089B0044623B9A94940F2C120FAF79EFEB4
:1093C800162200210DF10A0001F018FEA44EA5494D
:1093D80022788DF80820761AF608012336048DF8CD
:1093E800093046F004051F460C2A00F24B82DFE8DC
:1093F80012F00D00B0009A00B000B0004902B000B1
:109408009F00B000920026003D00A700964928461C
:10941800FAF740FB8DF80C709DF80920934928460F
:10942800FAF73CFBD4E9011302A898479DF80930E4
:10943800012B00F012828E4B05201B680CE28D492F
:109448002846FAF727FB4FF08053D3F80021039200
:10945800D3F804210492D3F80C2192020692D3F88F
:109468001021920205921B690793D5E78249834E22
:109478002846FAF70FFB227C81492846FAF70EFBAB
:1094880043F20403326A18687E4988420CBF0223FB
:109498000123012A4FF001028DF80920227C08BF20
:1094A800013352B902238DF80C30F3680493764BDC
:1094B8000593C3F5FC230693AEE7012A14D188422D
:1094C80012D100234FF440528DF80C301278142A30
:1094D80084BF43F214031B6804934FF4805305932D
:1094E80043F208031B68E6E79A4209D201238DF884
:1094F8000C30B368049300F0ABFCB3690590DAE76D
:1095080062492846FAF7C6FAFF238DF80C30002383
:10951800CDE90433CFE75E492846FAF7BBFA237C46
:109528008DF80C3078E75B492846FAF7B3FA73E709
:1095380059492846FAF7AEFA238AADF80C306BE79A
:1095480028465649FAF7A6FA494B07201B68984758
:1095580062E7062A524F01D0012A01D123693B70E4
:109568003B78012B0AD0022B00F0AE804D4946F023
:109578000100FAF78FFA00233B7000E1013A072A4D
:1095880066D8DFE802F004651444655D651E464947
:109598002846FAF77FFA364B03201B68984760691C
:1095A80000F04CFEFFF794FE8DF8090034E73F49C0
:1095B8002846FAF76FFA314BDA6B1B6C0392049367
:1095C8002AE7236923B925494FF48770FAF796FDEE
:1095D800A38A23B9214940F20F10FAF78FFD3449C5
:1095E8002846FAF757FAA18A206900F043FEFFF7E8
:1095F8006FFE224B8DF80900DA6B1B6C0493E3684D
:109608000392002B3FF408AF2069984704E72949E3
:109618002846FAF73FFA2849284800F061FEFFF784
:1096280057FE01288DF809007FF4F6AE002000F0FF
:10963800F9FA08B9224977E70A238DF80930EBE6E9
:1096480020492846FAF726FA4FF480730593B2E7C3
:10965800024940F27310FAF751FDDDE678CE0700B3
:109668004CB1070024B10700C5CE0700E6D30700B8
:10967800D0590020E8CE07000BCF0700445D00203A
:109688002ECF0700DBE5B151003007004BCF0700B4
:1096980062CF070079CF07009DCF0700B7CF07003B
:1096A8003C2000204FD30700CFCF0700F9CF070099
:1096B8001DD0070046D00700C8590020CC5900200B
:1096C80071D0070096D00700013A072A00F2D68029
:1096D800DFE812F00800D4009700A600D400C50007
:1096E800D40060006B492846FAF7D4F900F0F2FD7F
:1096F80030B9694946F00100FAF7CCF908239CE72C
:10970800626932B9654946F00100FAF7C3F90323E3
:1097180093E7C2F30B0343B1614B62495B6D096880
:1097280013448B4201D06049EDE7B2F5805F06D95A
:109738005E4946F00100FAF7ADF904237DE7584F7A
:1097480058497B6D0968D018884206D9009146F0BF
:1097580001005749FAF7B6F9D0E77A64FA6CBA64A7
:10976800544A3B6510683B63002201211844FFF707
:109778000FFD30B1504946F00100FAF78BF9052387
:109788005BE7BB6C00933B6D7A6C4C492846FAF753
:1097980099F941E64A492846FAF77CF900F09AFD1A
:1097A8000028ABD03E4FD7E914329B1AA28A134443
:1097B8007A6C934201D94349A5E73E4B3E6B1B683F
:1097C8001E44E36823B940494FF4F370FAF796FC56
:1097D800E368A28A21693046FFF79CFC08B1E36878
:1097E80012E7A18A3B6B394A20690B443B633B6D06
:1097F8000B443B65FAF764FC3B6DB8640490039333
:109808000AE6274E32492846FAF744F9B36C326D16
:1098180030492846FAF74CF9B36C0493336DEEE7F8
:1098280028462D49FAF736F91D48D0E91473426CD9
:10983800FB1A934205D0294946F00100FAF738F996
:109848005CE7836CC3640021416447652046FFF7E9
:1098580047FD234B1B680420984709B0F0BD2149F8
:109868002846FAF717F90E4B4FF480519A6C1B6D86
:1098780005910091049203931B4987E7124940F22E
:109888008920E8E6194946F00300FAF707F90223A8
:10989800D3E600BFC0D00700E7D007001CD10700FF
:1098A800445D0020C859002035D1070056D1070073
:1098B8007AD10700CC590020EBD1070002D207006B
:1098C8003DD2070063D2070078CE07008C5D0020E8
:1098D8007AD207009BD20700B1D20700D9D207007D
:1098E800D0590020FDD2070024D307006FD307000A
:1098F800836810B58BB10A4A1821FAF7EBFA0446C7
:1099080048B10848084B0949C01AC008000440F08B
:109918000200FAF7BFF8204610BD0724FBE700BF96
:10992800B59307004CB1070024B107005CCE0700CF
:1099380038B50546C0B10120FFF7C4FB044648B955
:1099480000F048FC00F0C6FC30B9084B00201D6050
:10995800FFF754FC204638BD0549064800F0C0FC16
:109968000128F2D00324F5E70724F3E7D0590020B3
:10997800C8590020CC5900202DE9F04716464FF46D
:10998800DC721F46054688461E4C01F0D8FA1E4B6D
:10999800E41AE408240444F0040A814650B91B4937
:1099A8005046FAF777F816B90020BDE8F087484620
:1099B800B047F9E716495046FAF76CF82A461549B0
:1099C8005046FAF76BF8002201212846FFF7E0FB22
:1099D80030B1114944F00100FAF75CF80320E4E7DC
:1099E8004FF4DC724146384601F0DFFA33464FF453
:1099F800DC7239462846FFF78DFB0028D4D007498A
:109A0800E8E700BF54B1070024B10700AED607004D
:109A1800F8D607000CD707002CD707004FD7070048
:109A280010B5084C2368013309D000225821201DA5
:109A3800FAF746FB23681B1A5842584110BD00200C
:109A4800FCE700BF00F0070070B5084C054600228F
:109A58005821201DFAF734FB2A4620602146044B82
:109A68000448BDE87040FFF787BF00BF445D002091
:109A7800D459002000F007002DE9F0473D4B3E4C3B
:109A88003E49E41AE408240444F0040A0546504612
:109A9800FAF700F82846FFF715FB054648B138499C
:109AA800024644F00100F9F7F9FF03252846BDE80E
:109AB800F087344FFFF7B4FFD7F80090D9F800309B
:109AC80001330646B8463AD02A46582109F104001F
:109AD800FAF7F6FAD9F80030834230D146B92A4964
:109AE80044F00300F9F7D6FF4FF4DC7239681AE046
:109AF800D8F8000025495422043001F020FA06461F
:109B0800D8F8000022494FF480725C3001F017FA4F
:109B180006B9A8B11F4944F00200F9F7BBFFD8F80D
:109B280000104FF4DC721C4801F03FFA0020FFF7E8
:109B38008BFF05460028B9D002461849B1E756B14F
:109B480050461749F9F7A6FF4FF4DC721549124839
:109B580001F02BFAAAE7104D134944F00200F9F777
:109B680099FF4FF4DC723146284601F047FA012389
:109B78006B60DBE724B1070054B1070056D4070037
:109B880079D407004020002034D5070004F00700EE
:109B98005CF00700A4D40700445D00200DD5070041
:109BA800F1D5070000F007008DD50700F8B5134B75
:109BB800134C144DE41AE408240407460E462A6898
:109BC800114944F00300F9F769FFFFF729FF20B9AD
:109BD8000E4940F26110FAF791FA3A460C4B2868A0
:109BE8003146FFF7C9FE024630B144F00100094989
:109BF800BDE8F840F9F752BFF8BD00BF24B107002F
:109C080054B1070040200020FDD5070027D60700E3
:109C18008C5B002071D607000149FFF7C7BF00BF62
:109C280000F0070038B505460020FFF70DFF044691
:109C380018B903492846FFF7B9FF204638BD00BFC9
:109C4800445D002029DF704738B50C4D0446D5F82F
:109C58009C3178B101330FD1002218210430FAF772
:109C68002FFA21462060072205F5CE70BDE838405E
:109C7800FFF7E8BF0E2038BD0820FCE700F007001A
:109C880008B528B11C22034901F08FF9002008BD4E
:109C98000E20FCE79CF1070010B5064C00221821A5
:109CA8002046FAF70DFA54F8043C1B1A584258415A
:109CB80010BD00BFA0F1070008B50F4BD3F85C2119
:109CC800013203D1D3F89C31013313D00B4B0C482C
:109CD8000C49C01AC008000440F00400F9F7DAFE85
:109CE8004FF4FE20FBF742FB572203494FF4FE20B6
:109CF800FBF754FB002008BD445D002024B1070099
:109D08005CB1070087D707002DE9F843144B154CC1
:109D1800DFF86090144D1549E41AE408A5EB09052D
:109D28002404ED0844F0040407462A462046F9F7BF
:109D3800B5FE0026AE4202D14FF000080BE059F8FC
:109D4800363038469847804640B10346324608497F
:109D58002046F9F7ADFE4046BDE8F8830136E9E74D
:109D680024B1070024B1070018B1070013D8070071
:109D780037D8070010B107002DE9F843154B164CEA
:109D8800DFF86490154D1649E41AE408A5EB0905B7
:109D98002404ED0844F0040407462A462046F9F74F
:109DA8007DFE0026AE4202D14FF000080CE009EB20
:109DB800C60338465B689847804640B1034632463A
:109DC80008492046F9F774FE4046BDE8F883013695
:109DD800E8E700BF24B1070024B1070018B1070065
:109DE800C4D70700E9D7070010B1070008B50C224F
:109DF800002101F003F9024B00221A6308BD00BFDD
:109E0800445D002043F204031A68084B9A4201BFDC
:109E180043F20803186800F6FF7020F47F600CBF57
:109E280020F00F004FF48050704700BFDBE5B151C0
:109E380008B5FFF7E7FF054B9B69184400F6FF706C
:109E480020F47F6020F00F0008BD00BF445D0020B3
:109E5800FFF7D8BF4FF4805070470000F8B5174B94
:109E6800174C184E1849E41AE408240444F0040472
:109E780005462046F9F70EFE376A012F06D013492A
:109E88002046F9F707FE00252846F8BD85B1F36995
:109E980073B1FFF7B7FF0022B169FAF711F9F36957
:109EA800834205D03A460A492046F9F7F7FDEBE721
:109EB80008492046F9F7EEFD0125E5E724B107003A
:109EC80024B10700445D002063D807007ED807004E
:109ED80094D80700B7D807002DE9F04F89B0074696
:109EE80001920593714A724B04919B1ADB081B047B
:109EF80043F004046F4902932046F9F7CBFD3A4634
:109F08006D496E4E6E4DDFF804922046F9F7C6FD96
:109F1800049B6C49002B0CBF32462A462046F9F7B1
:109F2800BDFD019B6849002B0CBF32462A462046DE
:109F3800F9F7B4FD059B6549002B0CBF32462A464C
:109F48002046F9F7ABFD43F2040361491A68614BF7
:109F580020469A4214BF32462A46F9F79FFD5E49C9
:109F68002046F9F797FDD9F81830D9F820205B4931
:109F78002046F9F79DFDD9F82430D9F82C20584906
:109F88002046F9F795FD4FF00008CDF81890B34634
:109F9800AA465FFA88F9B9F1010F51D0B9F1020F59
:109FA8005DD0FFF745FF019A0346002A46D0069A7E
:109FB800156A6A1E554255414A4E9E4205D24A4983
:109FC8000393CF20FAF79AF8039B0793F61A049B9A
:109FD8004649BE4238BF0123424620460393F9F75B
:109FE8005DFD079B42491A462046F9F757FDBE42D8
:109FF8002CBF5A4652463F492046F9F74FFD002DDF
:10A008000CBF5A4652463C492046F9F747FD039B88
:10A018003A49002B0CBF5A4652462046F9F73EFDF6
:10A02800039B03B3FDB9B8F1020F04D008F101088E
:10A03800B8F1030FADD1BE4217D323E0019DBBE7B2
:10A04800FFF7E0FE059A03463AB943F204021568A1
:10A05800204AAD1A18BF0125AEE74D46ACE70125E9
:10A068004FF48053A8E7BE4209D2029B244943F02B
:10A078000200F9F70FFD042009B0BDE8F08FB9F12F
:10A08800000F06D020461F49F9F704FD1E48FFF7C8
:10A09800ADFE1E4D0024012305F12400C5E904434B
:10A0A800FFF7A4FE6F622046E6E700BF24B1070071
:10A0B80024B10700D2D80700F0D807000AD9070052
:10A0C80005D9070010D9070021D907002FD90700A3
:10A0D80044D90700DBE5B15154D9070063D907001B
:10A0E80083D9070000000700A3D90700EAD90700B1
:10A0F800F4D9070009DA07001EDA070031DA070089
:10A1080042DA07006EDA07005C5D0020445D00203B
:10A1180030B51449144C8A6B85B06D465C312846BD
:10A12800FBF70EFB95E80F0084E80F000F4B104A71
:10A13800E360002313600F4A0F49136020460F4A5B
:10A14800FBF79DFD044648B90D480E4B0E49C01A51
:10A15800C008000440F00100F9F79CFC204605B057
:10A1680030BD00BF445D00203C61002095A1070080
:10A178009C5F0020985F0020C0C60700C05F0020D9
:10A1880064B1070024B1070007DF07005B689A681D
:10A198000A4B9A4211D1D0E90132094909480133E1
:10A1A8000B60094B0949013A1A60094BC01AC008EB
:10A1B800000440F00400F9F771BC704744C607007A
:10A1C8009C5F002064B10700985F0020EADE07006A
:10A1D80024B1070030B5134D134CAB6B91B0FBB1F4
:10A1E800FFF796FFE0B16B6AD3B101232370FBF749
:10A1F8008BFF18B10D49B020F9F780FF20220C49D8
:10A208006846FBF7D1FF40236A460A490A48FBF72C
:10A21800D3FE18B10549BB20F9F770FF11B030BD66
:10A228000023E3E7445D0020D461002080DA0700C2
:10A2380070BD07004C610020E0BB070038B505463B
:10A2480078B1B0F5807F0ED8084C094B0021202248
:10A2580004F138001970216300F0D0FEA5630120D5
:10A2680038BD0320FCE70420FAE700BF445D002066
:10A27800D461002070B5134C0646E06BA36B4218FE
:10A288009A420D460BD9104B10481149C01AC00804
:10A29800000440F00100F9F7FDFB032070BD5C30BD
:10A2A8000A462044314600F080FEE36B04F1400288
:10A2B8002B4429463046E363F9F702FF2064012066
:10A2C800ECE700BF445D002024B1070064B107003B
:10A2D800CCDA0700014B1878704700BFD461002022
:10A2E8002DE9F04F8B4CD4E90E329A4287B0834661
:10A2F8008A460ED0884B89488949C01AC00800048C
:10A3080040F00100F9F7C6FB0825284607B0BDE86C
:10A31800F08F844B03931A7842B1FFF789FDCBF88D
:10A328000000636ACAF800300125EEE7FFF7F0FE87
:10A33800794C7A4B002800F0E3807B4A92F89C50D5
:10A348001DB91178002900F0DB800021CBF800103E
:10A35800CAF80010BDB1754D92F83881A5F199067B
:10A368001C1BE408240444F00307202270490592CA
:10A378003846F9F78FFB4DB96E4944F00200F9F7FA
:10A3880089FB1325C1E7A8466B4EE9E7B8F1000F32
:10A3980005D06A493846F9F77DFB1625B5E7DFF899
:10A3A800F0816749D8F800203846F9F777FB05AB04
:10A3B8000193644A644B0093D8F8003012686349EB
:10A3C8006348FBF787FE00286AD195F80080B8F14A
:10A3D800400F65D1DFF8BC914246691C484600F041
:10A3E800E4FD5C493846F9F755FB20214846FBF760
:10A3F800E8FE554A059B58495848CDE90098FBF7AF
:10A40800F7FD024640B344F00100554944F0040406
:10A41800F9F744FB53492046F9F73CFB42464946C5
:10A428002046F9F779FB50492046F9F733FBBDF888
:10A43800142045492046F9F76FFB4C492046F9F7A7
:10A4480029FB42464A492046F9F766FBF9F794F991
:10A458000028FBD1052558E746493846F9F71AFB85
:10A46800301D00F0DBF9012805467FF44EAF039B51
:10A47800187096F85930ABB996F8682092B1F06E1A
:10A4880088B30022CAF8000001231146FFF724FD13
:10A4980058B3394944F00100F9F7FCFA042534E7C8
:10A4A8000A2532E713F0010003D096F85A0000B1EC
:10A4B800F06D9B07E4D596F86030002BE0D02F4B69
:10A4C800726EC3F5FC239A4201D81044D8E72C4990
:10A4D80044F00100F9F7ECFA04252A4944F0010098
:10A4E800F9F7D8FA11E70F25F7E7FFF7A1FC264996
:10A4F800CBF80000024644F00400F9F7CFFA04E76D
:10A50800181BC0080004214940F00100F9F7C2FAFD
:10A51800A0E700BF445D002024B1070064B1070034
:10A52800EFDA0700D4610020C05F0020F960002046
:10A538000ADB070032DB0700C45F002046DB0700A8
:10A548005DDB07009C5F0020A05F0020E4C50700DA
:10A55800205F002090DB07004C610020D8610020BC
:10A56800A1DB0700C3DB0700CEDB0700D4DB070055
:10A5780070BD0700E0DB07003DDC07000030070086
:10A58800EFDB07000CDC070058DC070074DC070071
:10A59800985F0020946100202DE9F04F864B874C8E
:10A5A80093F89C20DFF870A203F1A4050833002A71
:10A5B80008BF1D468DB0202605F16F0B074689465A
:10A5C8003246594604A80396FBF7D2FD7C4B7D49D9
:10A5D800E41AE408240444F004084B463A4640468A
:10A5E800F9F766FA03AB01933A46CDF800A04B465B
:10A5F80075497648FBF76EFD024648B1744944F048
:10A608000100F9F74BFA17247248FFF7EFFB53E004
:10A61800324604A9504600F092FCD8B16E4944F085
:10A628000200F9F737FA6D494046F9F733FA32462E
:10A6380059464046F9F770FA69494046F9F72AFA47
:10A64800324651464046F9F767FAF9F795F8002877
:10A65800FBD1D8E795F855A0624EBAF1000F17D094
:10A668001AF0010F0AF0020800F0A38042F2040376
:10A67800F95803F1A34303F5471303F2D75399425B
:10A688002CD0594944F00100F9F704FA0524BBE736
:10A6980001235649F3624046F9F7FCF995F88F30E3
:10A6A800C6F820A013B195F890300BB96B68B36069
:10A6B800B36CC6E909930124202200214C4800F01C
:10A6C8009DFCF422FF214B4800F098FC454B0022EA
:10A6D80020461A639F640DB0BDE8F08FAB6D03F59B
:10A6E800FF5203F6FF731F32C3F30B03D31A42F270
:10A6F8000802BA589A4201D23F49C3E743F2040319
:10A708001B688B4214BF4FF0010A4FF0000A29D191
:10A718004FF4405307F500521B781278142B81BF71
:10A7280043F2140335481B68B3FBF0F398BF0346A4
:10A73800142A81BF42F214023049BA58B2FBF1F22E
:10A7480098BF00222E490092934244F003002D4AFC
:10A7580018BF0A462C4914BF4FF0010A4FF0000AEF
:10A76800F9F7B0F9BAF1000F1DD0284944F00200FA
:10A77800F9F790F9B8F1000F01D1254982E725488A
:10A78800FFF734FBAC23F362AB6D7363B8F1000FD2
:10A798008ED095F88F301BB195F89030002B87D16B
:10A7A8006B68F36084E7B8F1000F14BFAC23A523EE
:10A7B800E9E7AA23F362E9E7C05F002064B1070074
:10A7C80024B107009DDC0700E4C50700205F0020D6
:10A7D800D9DC0700685D00200ADD070024DD0700DA
:10A7E80036DD0700445D00206EDD070046DD07000A
:10A7F8007C5D0020A05D0020BFDD070040420F0007
:10A8080091DC070097DC070028DE070068DE0700F8
:10A81800A9DE07005C5D0020FC5E0020F8B5044658
:10A8280018B95549A220F9F769FC94F854309BB13E
:10A8380094F8550003280FD894F86D30032B17D0DF
:10A848004E4B4F484F49C01AC008000440F0010061
:10A85800F9F720F91420F8BD4948484B4A49C01A6D
:10A86800C008000440F00100F9F714F90F20F2E7DE
:10A8780094F88F301BB194F89030002B79D1237A5B
:10A8880033B93F483D4B4149C01AC0080004E9E7C5
:10A89800E368342B0BD0394B39483D49C01AC008FE
:10A8A800000440F00200F9F7F5F81120D3E743F26D
:10A8B8000402237C1168374A914244D1002B36D0D8
:10A8C8006269002A33D004F11405002243F20C0611
:10A8D800D1B28B420BD8294B29482F49C01AC0083E
:10A8E800000440F00200F9F7D5F81220B3E755F854
:10A8F800227031888F4202F10102E9D12378002BBE
:10A908002DD001286368254A23D89268934234BF22
:10A91800002301236BBB194B19482149C01AC008F1
:10A92800000440F00200F9F7B5F8102093E728B9C1
:10A93800012BE3D96369002BE0D1CCE710F1FF3399
:10A9480018BF0123F7E713B16369002BC3D123783C
:10A95800F1E7D268934294BF00230123DAE7012884
:10A968003FF479AF0648054B0E49C01AC0080004E9
:10A9780078E701206FE700BF47DF070024B1070031
:10A988006CB10700AEDF070097DF0700C1DF0700E3
:10A99800D0DF0700DBE5B151E3DF0700445D0020AD
:10A9A800F3DF070007E0070010DF704711DF70478B
:10A9B80013B5044609496846FAF7F6FA019808B942
:10A9C80002B010BDD0E900312046984718B168465A
:10A9D800FAF704FBF2E71120F2E700BF38E00700BE
:10A9E80013B5044607496846FAF7DEFA019B0BB926
:10A9F80002B010BD2046D3E9002190476846FAF717
:10AA0800EDFAF3E750E00700064B9A6822B11A689E
:10AA180022F480021A607047034B4FF48002C3F897
:10AA2800802070473C32002000E100E00B4991F89B
:10AA380016335A09EC231341DB0706D5084B9A68ED
:10AA48003AB94FF480030B60704742F20200FBF7FB
:10AA580023BC1A6842F480021A60704700E100E0E3
:10AA68003C320020F7B5184F3C785CBB174E0125E7
:10AA780020463570FFF79CFF112820D02046FFF7AD
:10AA8800AFFF134B1868019002A800F8054DF9F7BD
:10AA9800C7FA104901A8FFF787FF0446B0FA80F00B
:10AAA800400938709DF80300F9F7EAFA3CB90A4BF7
:10AAB80034701C70FFF7BAFF2846FFF791FF204655
:10AAC80003B0F0BD0824FAE7DD610020DC61002056
:10AAD80032E0070075620700DE610020F7B5154F08
:10AAE8003B7813B3144E01203070FFF761FF112833
:10AAF8004FF000051BD00220FFF772FF02A800F8F4
:10AB0800015DF9F78DFAFFF751FF04469DF807003C
:10AB18003D70F9F7B5FA2CB93470FFF775FF0320CB
:10AB2800FFF75EFF204603B0F0BD0824FAE72C4685
:10AB3800F8E700BFDD610020DC610020054B1B78D1
:10AB480033B1054B1B780BB1FFF7C8BFFFF78ABFBE
:10AB580008207047DC610020DD610020014B187877
:10AB6800704700BFDD61002007B508496846FAF75D
:10AB78001BFA019B13B903B05DF804FBD3E900206D
:10AB880090476846FAF72AFAF3E700BF44E007005F
:10AB9800FFF7EABF60DF704769DF704761DF704722
:10ABA80030B5114DADF5017D4FF4FA740DF1020188
:10ABB80003A8ADF80240FFF7F1FF70B9294601A8D4
:10ABC800FAF7F2F9029B002BF0D003A8D3E9002191
:10ABD800904701A8FAF702FAF4E7052801D0FBF735
:10ABE8005BFB0DF5017D30BDD4E20700024B1B78FD
:10ABF8000BB1FFF7D5BF7047DF61002018B1034BD9
:10AC08000360002070470E20704700BFF01F00202F
:10AC180030B5054685B00C46002900F0B5805B4B81
:10AC28000B600C22002101A800F0E8F901238DF83F
:10AC3800063022688DF80450062301A92020ADF8BB
:10AC48000830FFF7A9FF60B1FAF702FA504A514BF2
:10AC580051499B1ADB081B04024643F00100F8F730
:10AC68001DFF0C22002101A800F0C8F901238DF86E
:10AC780005302268002301A940208DF806308DF8A0
:10AC88000730FFF789FF60B1FAF7E2F9404A414B14
:10AC980042499B1ADB081B04024643F00100F8F7FF
:10ACA800FDFE0C22002101A800F0A8F9F723226874
:10ACB8008DF8045001A92320ADF80630FFF76CFF8A
:10ACC80060B1FAF7C5F9324A324B35499B1ADB08AD
:10ACD8001B04024643F00100F8F7E0FE0C220021B5
:10ACE80001A800F08BF9012022688DF8040001A961
:10ACF800FFF752FF60B1FAF7ABF9254A254B29490E
:10AD08009B1ADB081B04024643F00100F8F7C6FE55
:10AD18000C22002101A800F071F94FF4B0632268F9
:10AD2800019301A9A120FFF737FF60B1FAF790F965
:10AD3800174A184B1C499B1ADB081B04024643F0B0
:10AD48000100F8F7ABFE0C22002101A800F056F92B
:10AD58009DF80430226843F0010301A9A0208DF872
:10AD68000430FFF719FF68B1FAF772F9084A094B7E
:10AD78000E499B1ADB081B04024643F00100F8F752
:10AD88008DFE002005B030BD0E20FBE7F01F00202F
:10AD980024B1070084B1070064E00700AAE00700B7
:10ADA800F6E007003DE1070089E10700DAE1070066
:10ADB800F8B506460768FFF7EDFE3368BB4205465F
:10ADC8001DD9194B194C1A49E41AE408240444F013
:10ADD80002042046F8F75EFE336816493A462046D4
:10ADE800F8F766FE4FF080533268D3F80C311249F9
:10ADF8009B0203F100539A1A2046F8F74FFE25B933
:10AE08000E4B01221A702846F8BD2846FAF720F999
:10AE1800054A064B0A499B1ADB081B04024643F005
:10AE28000100F8F73BFEEEE724B1070084B1070004
:10AE38002DE207005CE207008DE20700DF610020D9
:10AE4800B7E207004BDF70471FB50D4C01A8FFF7AD
:10AE5800F9FF70B9214602A8FAF7A6F8039B002B60
:10AE6800F4D00198D3E90021904702A8FAF7B6F880
:10AE7800F4E7052801D0FBF70FFA04B010BD00BFB6
:10AE8800ECE207007F2805D8034B185C034B5B5C9A
:10AE9800184070470020704704E3070084E3070068
:10AEA800A0F16103192B98BF20387047A0F1410326
:10AEB800192B98BF203070477F2805D8034B185CA2
:10AEC800034B5B5C184070470020704704E30700A1
:10AED80084E30700A0F16103192B98BF203870475D
:10AEE800A0F14103192B98BF203070477F299ABFE2
:10AEF800017001206FF02E0070475AB10A787F2A3E
:10AF08000AD800B10260002119605960501A18BFB0
:10AF180001207047002070476FF02E007047000036
:10AF280008B5034B5B689B681B68984708BD00BF62
:10AF38004420002008B50921FFF7F2FF08BD92B3AD
:10AF480070B4134640EA010212F0030F17D05A1EDC
:10AF580010D004780B789C420CD1431C4C1C024442
:10AF680018462146934205D00133013406780D78FE
:10AF7800AE42F5D000780B78C01A70BC70470F2B22
:10AF8800E5D904680A689442E1D1041D0A1D2046E7
:10AF98001146043B042BDAD90434043206680D68E0
:10AFA800AE42F4D0D3E700207047844640EA01035C
:10AFB80013F0030F18D18446202A0BD32DE9F0078C
:10AFC800B1E8F807A0E8F807A2F12002202AF7D292
:10AFD800BDE8F007042A07D351F8043B40F8043BC6
:10AFE800A2F10402042AF7D2002A05D011F8013B85
:10AFF80000F8013B013AF9D1604670478446002ABF
:10B008002DD010F0030F04D000F8011B013A26D010
:10B01800F7E7C9B241EA012141EA0141202A12D3E6
:10B02800A2F120022DE9F0030B460C460D460E4610
:10B038000F4688468946A0E8FA03203AFBD2BDE8C5
:10B04800F00320320BD0042A05D340F8041B043A3D
:10B0580005D0042AF9D200F8011B013AFBD1604659
:10B068007047024610F0030F16D111F0030F13D1E9
:10B078002DE9F0004FF001374FF0803351F8044BC1
:10B08800A4EB070525EA04051D4002D142F8044B4C
:10B09800F4E7A1F10401F0BC11F8013B02F8013B0F
:10B0A800002BF9D1704700F1010110F0030F11D006
:10B0B80010F8012B002A23D010F0030F0AD010F843
:10B0C800012B002A1CD010F0030F03D010F8012B1D
:10B0D800002A15D02DE970004FF001324FF080336F
:10B0E80050F8044BA4EB020525EA04051D4000D1E5
:10B0F800F6E7A0F1040070BC10F8012B002AFBD180
:06B10800A0EB01007047FE
:08B11000AD8E07006D8B0700F6
:0CB118000000000003000000895E07003A
:10B12400E1B2070000000404F2B3070000000000CD
:10B13400C0C507000000040490CC0700000004040C
:10B1440032CE07000000040442D4070000000404C7
:10B1540076D7070000000404AED7070000000404FB
:10B1640034DF0700000004041BE0070000000404AF
:10B17400F2B40700000004045CE0070000000303CD
:10B18400E0E2070000000303F8E207000000030305
:10B194009C200020642100206C210020A420002099
:10B1A40018000000304900206C5900207D5900200F
:08B1B40038490020F4000000FE
:08B1BC005986070000000000A5
:10B1C40018B20700000000006FB20700042000203E
:10B1D400F5AB07000000000051AE070000000000BE
:08B1E400514B070000000000C0
:08B1EC00114D070000000000F6
:08B1F4006D4C07000000000093
:10B1FC000000000000000000459007000010000057
:04B20C000000080036
:10B210000338FDD870470000DD33070049340700CC
:10B22000D9330700433A2F6E5246355F53444B5F84
:10B2300031352E322E302F636F6D706F6E656E74E8
:10B24000732F6C69627261726965732F6C6F672FFF
:10B250007372632F6E72665F6C6F675F64656661A1
:10B26000756C745F6261636B656E64732E630072EC
:10B2700074745F6C6F675F6261636B656E640043DB
:10B280003A2F6E5246355F53444B5F31352E322E86
:10B29000302F636F6D706F6E656E74732F6C6962A3
:10B2A0007261726965732F6C6F672F7372632F6E93
:10B2B00072665F6C6F675F66726F6E74656E642E28
:10B2C00063000000903100207F0000001032002059
:10B2D0004261636B656E647320666C757368656448
:10B2E00000617070000000001BB3070060B307002E
:10B2F00020B3070068B3070070B3070078B30700F6
:10B3000080B3070088B3070090B3070020253032D0
:10B310007800202020007C002563001B5B306D003E
:10B320001B5B313B33316D0025734C6F67732064B9
:10B33000726F70706564202825642925730D0A00DA
:10B340003C25733E2025733A2000000000000000D9
:10B3500098B307009EB30700A6B30700ABB307007E
:10B360001B5B313B33306D001B5B313B33326D0077
:10B370001B5B313B33336D001B5B313B33346D0062
:10B380001B5B313B33356D001B5B313B33366D004E
:10B390001B5B313B33376D006572726F72007761F2
:10B3A000726E696E6700696E666F006465627567CC
:10B3B00000433A2F6E5246355F53444B5F31352E72
:10B3C000322E302F636F6D706F6E656E74732F6CDD
:10B3D00069627261726965732F7574696C2F61702F
:10B3E000705F7574696C5F706C6174666F726D2EDE
:10B3F00063006D656D5F6D6E677200433A2F6E522C
:10B4000046355F53444B5F31352E322E302F636FFC
:10B410006D706F6E656E74732F6C696272617269A4
:10B4200065732F62616C6C6F632F6E72665F626111
:10B430006C6C6F632E6300433A2F6E5246355F5338
:10B44000444B5F31352E322E302F65787465726E25
:10B45000616C2F667072696E74662F6E72665F66BD
:10B460007072696E74662E63003031323334353653
:10B47000373839414243444546433A2F6E524635A8
:10B480005F53444B5F31352E322E302F6578746513
:10B49000726E616C2F667072696E74662F6E726662
:10B4A0005F667072696E74665F666F726D61742E2E
:10B4B0006300433A2F6E5246355F53444B5F31353C
:10B4C0002E322E302F636F6D706F6E656E74732F1A
:10B4D0006C69627261726965732F6673746F7261F1
:10B4E00067652F6E72665F6673746F726167652E33
:10B4F00063006E72665F6673746F726167650000E9
:10B50000001000000400000001000000E9490700ED
:10B510000D4A07001D4A0700894A07002D4A070007
:10B52000F5490700F9490700FD4907000010000030
:10B530000400000001000000954B0700754B070058
:10B54000654B07009D4D0700514D0700394B070023
:10B550003D4B0700414B0700433A2F6E5246355F83
:10B5600053444B5F31352E322E302F636F6D706F29
:10B570006E656E74732F6C69627261726965732F88
:10B580006D656D6F626A2F6E72665F6D656D6F625D
:10B590006A2E6300433A2F6E5246355F53444B5F29
:10B5A00031352E322E302F636F6D706F6E656E7475
:10B5B000732F6C69627261726965732F657870654B
:10B5C00072696D656E74616C5F73656374696F6ECB
:10B5D0005F766172732F6E72665F73656374696FF5
:10B5E0006E5F697465722E6300556E6B6E6F776E59
:10B5F000206572726F7220636F6465000000000046
:10B6000024B707000100000030B707000200000067
:10B610004EB70700030000006FB7070004000000EA
:10B6200082B707000500000093B70700060000007E
:10B63000A7B7070007000000BFB707000800000019
:10B64000D7B7070009000000EFB707000A000000A5
:10B6500008B807000B00000020B807000C0000002D
:10B6600037B807000D0000004BB807000E000000BF
:10B670005DB807000F0000006CB807001000000064
:10B6800080B807001100000097B807001200000002
:10B69000A6B8070013000000BBB807008000000038
:10B6A000CFB8070081000000F0B80700820000005A
:10B6B0000CB907008300000028B9070084000000CF
:10B6C00046B907008500000067B907008600000042
:10B6D0008CB9070090000000A3B90700910000009A
:10B6E000C1B9070092000000DFB907000082000026
:10B6F000F4B907000182000012BA070002820000BC
:10B700002EBA0700008400004ABA07000184000036
:10B710006EBA07000284000098BA07000384000094
:10B72000BDBA07004E52465F53554343455353003D
:10B730004E52465F4552524F525F5356435F484107
:10B740004E444C45525F4D495353494E47004E526B
:10B75000465F4552524F525F534F465444455649F7
:10B7600043455F4E4F545F454E41424C4544004E69
:10B7700052465F4552524F525F494E5445524E41D8
:10B780004C004E52465F4552524F525F4E4F5F4DF6
:10B79000454D004E52465F4552524F525F4E4F54F8
:10B7A0005F464F554E44004E52465F4552524F52EF
:10B7B0005F4E4F545F535550504F52544544004EC6
:10B7C00052465F4552524F525F494E56414C494492
:10B7D0005F504152414D004E52465F4552524F52CA
:10B7E0005F494E56414C49445F5354415445004EC5
:10B7F00052465F4552524F525F494E56414C494462
:10B800005F4C454E475448004E52465F4552524F9A
:10B81000525F494E56414C49445F464C41475300A4
:10B820004E52465F4552524F525F494E56414C4927
:10B83000445F44415441004E52465F4552524F527C
:10B840005F444154415F53495A45004E52465F455B
:10B8500052524F525F54494D454F5554004E524637
:10B860005F4552524F525F4E554C4C004E52465F10
:10B870004552524F525F464F5242494444454E0052
:10B880004E52465F4552524F525F494E56414C49C7
:10B89000445F41444452004E52465F4552524F521B
:10B8A0005F42555359004E52465F4552524F525FC8
:10B8B000434F4E4E5F434F554E54004E52465F45E8
:10B8C00052524F525F5245534F5552434553004ECB
:10B8D00052465F4552524F525F4D4F44554C455F63
:10B8E0004E4F545F494E495449414C495A454400D2
:10B8F0004E52465F4552524F525F4D555445585F28
:10B90000494E49545F4641494C4544004E52465FBA
:10B910004552524F525F4D555445585F4C4F434B23
:10B920005F4641494C4544004E52465F4552524F96
:10B93000525F4D555445585F554E4C4F434B5F46F3
:10B9400041494C4544004E52465F4552524F525F6A
:10B950004D555445585F434F4E445F494E49545FDF
:10B960004641494C4544004E52465F4552524F5263
:10B970005F4D4F44554C455F414C52454144595FE2
:10B98000494E495449414C495A4544004E52465F3C
:10B990004552524F525F53544F524147455F4655AF
:10B9A0004C4C004E52465F4552524F525F415049F7
:10B9B0005F4E4F545F494D504C454D454E544544A4
:10B9C000004E52465F4552524F525F4645415455D4
:10B9D00052455F4E4F545F454E41424C4544004EE8
:10B9E00052465F4552524F525F494F5F50454E4459
:10B9F000494E47004E52465F4552524F525F4452A5
:10BA0000565F5457495F4552525F4F564552525503
:10BA10004E004E52465F4552524F525F4452565F5F
:10BA20005457495F4552525F414E41434B004E527D
:10BA3000465F4552524F525F4452565F5457495FDA
:10BA40004552525F444E41434B004E52465F455271
:10BA5000524F525F424C455F495053505F52585FBE
:10BA6000504B545F5452554E4341544544004E523E
:10BA7000465F4552524F525F424C455F49505350CA
:10BA80005F4348414E4E454C5F414C5245414459FD
:10BA90005F455849535453004E52465F4552524FEA
:10BAA000525F424C455F495053505F4C494E4B5F8B
:10BAB000444953434F4E4E4543544544004E52462D
:10BAC0005F4552524F525F424C455F495053505F61
:10BAD000504545525F52454A454354454400000095
:10BAE000982F8A4291443771CFFBC0B5A5DBB5E9E9
:10BAF0005BC25639F111F159A4823F92D55E1CAB5D
:10BB000098AA07D8015B8312BE853124C37D0C55EA
:10BB1000745DBE72FEB1DE80A706DC9B74F19BC132
:10BB2000C1699BE48647BEEFC69DC10FCCA10C2422
:10BB30006F2CE92DAA84744ADCA9B05CDA88F97606
:10BB400052513E986DC631A8C82703B0C77F59BF70
:10BB5000F30BE0C64791A7D55163CA06672929149C
:10BB6000850AB72738211B2EFC6D2C4D130D385339
:10BB700054730A65BB0A6A762EC9C281852C7292FB
:10BB8000A1E8BFA24B661AA8708B4BC2A3516CC729
:10BB900019E892D1240699D685350EF470A06A1062
:10BBA00016C1A419086C371E4C774827B5BCB034B1
:10BBB000B30C1C394AAAD84E4FCA9C5BF36F2E684F
:10BBC000EE828F746F63A5781478C8840802C78CDE
:10BBD000FAFFBE90EB6C50A4F7A3F9BEF27871C6E1
:10BBE00048002800002040004D7007002958070039
:10BBF000CB5707001D5D07008F5D0700AF5D070095
:10BC00000D570700CD560700A55C07000000000097
:10BC1000433A2F6E5246355F53444B5F31352E32D7
:10BC20002E302F636F6D706F6E656E74732F626F41
:10BC3000617264732F626F617264732E63001112FC
:10BC40001314433A2F6E5246355F53444B5F3135E0
:10BC50002E322E302F6D6F64756C65732F6E726689
:10BC6000782F68616C2F6E72665F6770696F2E68DF
:10BC700000433A2F6E5246355F53444B5F31352EA9
:10BC8000322E302F636F6D706F6E656E74732F6C14
:10BC900069627261726965732F63727970746F2F54
:10BCA0006E72665F63727970746F5F7368617265DC
:10BCB000642E630052656365697665642061206661
:10BCC00061756C74212069643A20307825303878A9
:10BCD0002C2070633A203078253038782C20696E1B
:10BCE000666F3A2030782530387800526563656990
:10BCF00076656420616E206572726F723A203078CA
:10BD0000253038782100000000000000000000000D
:10BD10000338FDD8704740404040404040404040DC
:10BD20004040404040404040404040404040404013
:10BD30004040404040004254204156204150532B47
:10BD4000204446550020202020202020257300314B
:10BD50002E302E302E33313A6A6A31353438373747
:10BD600033313330004166746572206D61696E0055
:10BD700093CE9CB79E1F4D34F6BEBCAE4AA74DC4B1
:10BD800053D83962184A94A8B50D9DCA9195634954
:10BD9000DC9D645BFD6C847EDF60A2B86DB39D8129
:10BDA000FF7A687B4B1CC56C2A2B6EB9E7B66ADA42
:10BDB00008200001FFFFFFFFFFFFFFFFFFFFFFFF66
:10BDC0000000000000000000000000000100000072
:10BDD000FFFFFFFF512563FCC2CAB9F3849E17A77A
:10BDE000ADFAE6BCFFFFFFFFFFFFFFFF0000000012
:10BDF000FFFFFFFF96C298D84539A1F4A033EB2D81
:10BE0000817D0377F240A463E5E6BCF847422CE16C
:10BE1000F2D1176BF551BF376840B6CBCE5E316BB0
:10BE20005733CE2B169E0F7C4AEBE78E9B7F1AFE74
:10BE3000E242E34F4B60D2273E3CCE3BF6B053CCC0
:10BE4000B0061D65BC86987655BDEBB3E7933AAA5C
:10BE5000D835C65A176A07006D6B0700C96B070013
:10BE60005465726D696E616C0052545400534547BD
:10BE70004745520052756E6E696E67206E72665F3E
:10BE8000626F6F746C6F616465725F6170705F7315
:10BE90007461727420776974682061646472657378
:10BEA000733A203078253038780044697361626CC9
:10BEB000696E6720696E74657272757074732E2076
:10BEC0004E5649432D3E494345525B305D3A203042
:10BED000782578004661696C65642072756E6E69BC
:10BEE0006E67206E72665F6466755F6D62725F6911
:10BEF00072715F666F72776172645F6164647265AC
:10BF000073735F736574282900436F756C64206ECA
:10BF10006F742070726F7465637420626F6F746CDD
:10BF20006F6164657220616E642073657474696EFC
:10BF300067732070616765732C20307825782E0038
:10BF4000526573657474696E6720626F6F746C6F8D
:10BF5000616465722E000000000000000000000017
:10BF60000338FDD87047496E6163746976697479E6
:10BF70002074696D656F75742E00496E206E72664F
:10BF80005F626F6F746C6F616465725F696E697414
:10BF900000444655206D6F6465206265636175736A
:10BFA0006520617070206973206E6F742076616CFB
:10BFB00069642E00444655206D6F6465207265717A
:10BFC0007565737465642076696120627574746F39
:10BFD0006E2E00444655206D6F6465207265717544
:10BFE00065737465642076696120475052454752F5
:10BFF00045542E0053686F756C64206E65766572CB
:10C0000020636F6D6520686572653A2041667465CE
:10C010007220626F6F746C6F616465725F726573BA
:10C020006574282900456E746572206D61696E2003
:10C030006C6F6F7000433A2F6E5246355F53444B1E
:10C040005F31352E322E302F636F6D706F6E656EDF
:10C0500074732F6C69627261726965732F626F6F9E
:10C06000746C6F616465722F6E72665F626F6F745D
:10C070006C6F616465722E630053686F756C642029
:10C080006E6576657220636F6D6520686572653ACE
:10C09000204166746572206E72665F626F6F746CA9
:10C0A0006F616465725F6170705F73746172742830
:10C0B0002900696E207765616B206E72665F646629
:10C0C000755F696E69745F757365720074696D651B
:10C0D000725F73746F702028307825782900746936
:10C0E0006D65725F66697265202830782578290051
:10C0F0000338FDD8704774696D65725F6163746958
:10C10000766174652028307825782900433A2F6EAF
:10C110005246355F53444B5F31352E322E302F63FC
:10C120006F6D706F6E656E74732F6C696272617281
:10C130006965732F626F6F746C6F616465722F6EC7
:10C1400072665F626F6F746C6F616465725F646664
:10C15000755F74696D6572732E63005665726966EA
:10C1600079696E6720424C3A20416464723A20300B
:10C1700078253038782C205372633A203078253077
:10C1800038782C204C656E3A20307825303878008D
:10C19000436F7079696E6720626F6F746C6F616452
:10C1A00065723A205372633A203078253038782C03
:10C1B000204C656E3A20307825303878004E6F205C
:10C1C000626F6F746C6F6164657220636F70792049
:10C1D0006E65656465642C20626F6F746C6F61645A
:10C1E00065722075706461746520636F6D706C6535
:10C1F00074652E005265717565737420746F2063C9
:10C200006F707920424C206661696C6564004E6FE6
:10C2100020636F7079206E65656465642073726356
:10C220005F616464723A20307825782C20647374DE
:10C230005F616464723A203078257800433A2F6E4B
:10C240005246355F53444B5F31352E322E302F63CB
:10C250006F6D706F6E656E74732F6C696272617250
:10C260006965732F626F6F746C6F616465722F6E96
:10C2700072665F626F6F746C6F616465725F667720
:10C280005F61637469766174696F6E2E6300436FDA
:10C290007079696E67203078257820746F20307847
:10C2A00025782C2073697A653A2030782578004605
:10C2B00061696C656420746F2077726974652069A8
:10C2C0006D61676520636F7079696E672070726F4A
:10C2D000677265737320746F2073657474696E6719
:10C2E0007320706167652E00456E746572206E72F2
:10C2F000665F626F6F746C6F616465725F66775FB3
:10C3000061637469766174650056616C696420418B
:10C31000707000456E746572206E72665F6466753B
:10C320005F6170705F636F6E74696E7565005365F1
:10C330007474696E67206170702061732076616C1F
:10C3400069640043524320636F6D70757461746952
:10C350006F6E206661696C656420666F7220636F22
:10C3600070696564206170703A2073726320637233
:10C37000633A203078253038782C2072657320633A
:10C3800072633A203078253038780056616C6964E1
:10C390002053440056616C696420424C0056616C25
:10C3A0006964205344202B20424C00456E74657212
:10C3B000206E72665F6466755F73645F626C5F6354
:10C3C0006F6E74696E75650053442B424C3A20536E
:10C3D0004420636F7079206661696C656400534422
:10C3E0002B424C3A20424C20636F70792066616981
:10C3F0006C6564004E6F206669726D7761726520AE
:10C40000746F2061637469766174652E0041637492
:10C4100069766174696F6E206661696C6564207706
:10C42000697468206572726F7220256420286261C9
:10C430006E6B20636F64653A20307825782900415F
:10C4400020536F6674446576696365206861732064
:10C450006A757374206265656E20616374697661C4
:10C460007465642E2049742773206C696B656C7940
:10C47000207468617420616E206170706C69636102
:10C4800074696F6E2077696C6C20636F6D652069CD
:10C490006D6D6564696174656C7900436F756C647A
:10C4A000206E6F7420777269746520736574746987
:10C4B0006E67732E00456E746572206E72665F62E1
:10C4C0006F6F746C6F616465725F6466755F7364CF
:10C4D0005F636F6E74696E756500536F7572636527
:10C4E000206164647265737320646F6573206E6F7E
:10C4F0007420636F6E7461696E20612076616C696F
:10C500006420536F66744465766963652E005344F6
:10C5100020616C726561647920636F706965640085
:10C520005570646174696E672053442E204F6C64AB
:10C53000205344207665723A2025642C204E65777E
:10C54000207665723A202564004661696C65642036
:10C55000746F20636F7079206669726D77617265A0
:10C560002E0057445420656E61626C65642043520E
:10C57000563A2564207469636B7300537461727456
:10C58000696E6720612074696D65722028256420BA
:10C590007469636B732920666F72206665656469D0
:10C5A0006E67207761746368646F672E0057445428
:10C5B000206973206E6F7420656E61626C65640023
:10C5C0006E72665F626F6F746C6F616465725F77C5
:10C5D000647400496E7465726E616C206665656492
:10C5E000000000008B81070085810700658107003E
:10C5F000200000007800000000000000011101FF91
:10C600000100000000000000021702FE940000007C
:10C6100044C6070000000000000000000000000009
:10C620000101000001000000000000000205000000
:10C6300021000000000000000000000000000000D9
:10C6400000000000011104FC0400000000000000D4
:10C65000021104FC0400000000000000032104FC9F
:10C660000410000000000000041101FF01000000A0
:10C6700000000000051102FE0400000000000000A0
:10C68000061104FC0400000000000000071104FC77
:10C690000400000000000000081701FF2200000055
:10C6A00020C60700091001FF01000000BCC60700FA
:10C6B000000000000000000000000000000000007A
:10C6C000011704FC98000000FCC50700021704FCD9
:10C6D000DC000000E4C607000000000000000000CD
:10C6E000000000000107000098000000FCC50700E2
:10C6F000020100000100000000000000030500002E
:10C7000041000000000000000000000000000000E8
:10C7100000000000456E746572696E6720444655DE
:10C72000206D6F64652E00436F756C64206E6F74AE
:10C7300020696E6974616C697A652044465520747D
:10C7400072616E73706F72743A2030782530387869
:10C750000050EADA308883B89F604F15F30000C9B3
:10C760008E4164766572746973696E672E2E2E0031
:10C77000433A2F6E5246355F53444B5F31352E326C
:10C780002E302F636F6D706F6E656E74732F6C69D2
:10C79000627261726965732F626F6F746C6F61642E
:10C7A00065722F626C655F6466752F6E72665F647A
:10C7B00066755F626C652E63004446552072657134
:10C7C00075657374202564206661696C65642077E3
:10C7D000697468206572726F723A2030782578002B
:10C7E0005368757474696E6720646F776E20424C6D
:10C7F00045207472616E73706F72742E0044697399
:10C80000636F6E6E656374696E672E00424C4520DF
:10C810007472616E73706F727420736875742064C3
:10C820006F776E2E004466755461726700496E69B9
:10C830007469616C697A696E6720424C4520444690
:10C8400055207472616E73706F72740053657474E6
:10C85000696E6720757020766563746F72207461ED
:10C86000626C653A2030782530387800456E616218
:10C870006C696E6720536F66744465766963652ED4
:10C8800000436F6E6669677572696E6720424C453A
:10C8900020737461636B2E00456E61626C696E6714
:10C8A0002074686520424C4520737461636B2E00D0
:10C8B0004E6F206164766572746973696E67206E6D
:10C8C000616D6520666F756E640053657474696E82
:10C8D0006720616476206E616D653A2025732C2097
:10C8E0006C656E6774683A202564005573696E67DD
:10C8F0002064656661756C74206164766572746924
:10C9000073696E67206E616D6500424C4520444638
:10C9100055207472616E73706F727420696E6974E1
:10C9200069616C697A65642E00436F6E6E6563742D
:10C930006564004661696C75726520746F2075705E
:10C940006461746520636F6E6E656374696F6E20D9
:10C95000706172616D65746572733A203078257804
:10C960000063616E6E6F7420616C6C6F63617465DF
:10C97000206D656D6F727920627566666572210043
:10C9800042756666657220257020616371756972F3
:10C9900065642C206C656E202564202825642900A0
:10C9A000526563656976656420424C455F47415432
:10C9B00054535F4556545F45584348414E47455F81
:10C9C0004D54555F52455155455354202872657159
:10C9D000756573743A2025642C207265706C793A01
:10C9E000202564292E0052656365697665642042BE
:10C9F0004C455F4741505F4556545F444154415F49
:10CA00004C454E4754485F5550444154455F52454C
:10CA100051554553542E005265636569766564200F
:10CA2000424C455F4741505F4556545F4441544135
:10CA30005F4C454E4754485F55504441544520286B
:10CA400025752C206D61785F72785F74696D652043
:10CA50002575292E00526563656976656420424C10
:10CA6000455F4741505F4556545F5345435F5041D2
:10CA700052414D535F524551554553540043434332
:10CA80004420666F722073657276696365206368FF
:10CA9000616E6765642069732030782530347800D2
:10CAA000526563656976656420424C455F47415035
:10CAB0005F4556545F434F4E4E5F504152414D5F6C
:10CAC000555044415445006D61785F636F6E6E5FF1
:10CAD000696E74657276616C3A202564006D696ECA
:10CAE0005F636F6E6E5F696E74657276616C3A201B
:10CAF000256400736C6176655F6C6174656E637943
:10CB00003A20256400636F6E6E5F7375705F7469A1
:10CB10006D656F75743A20256400526563656976AA
:10CB2000656420424C455F4741505F4556545F4322
:10CB30004F4E4E5F504152414D5F55504441544518
:10CB40005F52455155455354004661696C75726595
:10CB500020746F2075706461746520636F6E6E65FC
:10CB60006374696F6E20706172616D6574657220A7
:10CB7000726571756573743A203078257800526556
:10CB800063656976656420424C455F4741505F4567
:10CB900056545F5048595F555044415445202852DF
:10CBA000583A25642C2054583A25642C207374611B
:10CBB0007475733A25642900526563656976656406
:10CBC00020424C455F4741505F4556545F5048599D
:10CBD0005F5550444154455F524551554553542E7D
:10CBE000005365742072656365697074206E6F749C
:10CBF000696600436F756C64206E6F742068616EA7
:10CC0000646C65206F6E5F6374726C5F70745F77C5
:10CC1000726974652E206572725F636F64653A2075
:10CC20003078253034780052656365697665642014
:10CC3000424C455F4741505F4556545F5345435F03
:10CC4000494E464F5F524551554553540046696E13
:10CC500069736865642068616E646C696E672063DF
:10CC60006F6E6E207365632075706461746500007B
:10CC70000338FDD870470C000C00000058024672C3
:10CC80006565696E6720627566666572202570004D
:10CC90006E72665F6466755F626C65007772697458
:10CCA0006500657261736500466C61736820257369
:10CCB00020737563636573733A20616464723D2504
:10CCC000702C2070656E64696E6720256400466C68
:10CCD000617368202573206661696C656420283063
:10CCE000782578293A20616464723D25702C206C87
:10CCF000656E3D307825782062797465732C2070DC
:10CD0000656E64696E67202564006E72665F667387
:10CD1000746F726167655F657261736528616464D1
:10CD2000723D307825702C206C656E3D2564207036
:10CD300061676573292C2071756575652075736150
:10CD400067653A202564006E72665F6673746F7261
:10CD50006167655F65726173652829206661696C2A
:10CD600065642077697468206572726F722030780C
:10CD700025782E00496E697469616C697A696E67FD
:10CD8000206E72665F6673746F726167655F73644D
:10CD9000206261636B656E642E00496E697469611F
:10CDA0006C697A696E67206E72665F6673746F7203
:10CDB0006167655F6E766D63206261636B656E644B
:10CDC0002E006E72665F6673746F726167655F775F
:10CDD0007269746528616464723D25702C207372D9
:10CDE000633D25702C206C656E3D2564206279744E
:10CDF0006573292C2071756575652075736167658C
:10CE00003A202564006E72665F6673746F726167A4
:10CE1000655F77726974652829206661696C65644D
:10CE20002077697468206572726F72203078257877
:10CE30002E006E72665F6466755F666C6173680073
:10CE400041667465722072756E6E696E67206972D4
:10CE500071207461626C652073657400536368654A
:10CE600064756C65722072616E206F7574206F66D8
:10CE70002073706163652100433A2F6E5246355F1F
:10CE800053444B5F31352E322E302F636F6D706FF0
:10CE90006E656E74732F6C69627261726965732F4F
:10CEA000626F6F746C6F616465722F6466752F6E4C
:10CEB00072665F6466755F7265715F68616E646CEF
:10CEC00065722E630048616E646C65204E52465F49
:10CED0004446555F4F505F50524F544F434F4C5F45
:10CEE00056455253494F4E0048616E646C65204E62
:10CEF00052465F4446555F4F505F48415244574148
:10CF000052455F56455253494F4E0048616E646C1E
:10CF100065204E52465F4446555F4F505F4649522A
:10CF20004D574152455F56455253494F4E00466951
:10CF3000726D7761726520696D61676520726571D8
:10CF40007565737465643A202564004E6F207375AF
:10CF50006368206669726D7761726520696D6167CB
:10CF6000650048616E646C65204E52465F444655CC
:10CF70005F4F505F50494E470048616E646C6520BA
:10CF80004E52465F4446555F4F505F5245434549B8
:10CF900050545F4E4F5449465F5345540048616EAC
:10CFA000646C65204E52465F4446555F4F505F4D5E
:10CFB00054555F4745540048616E646C65204E527D
:10CFC000465F4446555F4F505F41424F52540048C0
:10CFD000616E646C65204E52465F4446555F4F500B
:10CFE0005F4F424A4543545F4352454154452028D0
:10CFF000636F6D6D616E64290048616E646C6520BD
:10D000004E52465F4446555F4F505F4352435F4721
:10D0100045542028636F6D6D616E64290048616E10
:10D02000646C65204E52465F4446555F4F505F4FDB
:10D03000424A4543545F57524954452028636F6D17
:10D040006D616E64290048616E646C65204E5246C5
:10D050005F4446555F4F505F4F424A4543545F45DA
:10D060005845435554452028636F6D6D616E6429A2
:10D070000057726974696E672076616C6964206913
:10D080006E697420636F6D6D616E6420746F2066CD
:10D090006C6173682E0048616E646C65204E524668
:10D0A0005F4446555F4F505F4F424A4543545F537C
:10D0B000454C4543542028636F6D6D616E642900B3
:10D0C00048616E646C65204E52465F4446555F4F22
:10D0D000505F4F424A4543545F43524541544520B7
:10D0E0002864617461290043616E6E6F74206372FD
:10D0F000656174652064617461206F626A65637440
:10D1000020776974686F75742076616C6964206932
:10D110006E697420636F6D6D616E64004F626A6545
:10D1200063742073697A652063616E6E6F74206228
:10D130006520302E004F626A6563742073697A65DA
:10D14000206D757374206265207061676520616C65
:10D1500069676E656400496E76616C696420736905
:10D160007A6520666F72206F626A65637420287426
:10D170006F6F206C61726765290043726561746925
:10D180006E6720746865206F626A656374207769D2
:10D1900074682073697A6520307825303878207774
:10D1A0006F756C64206F766572666C6F7720666948
:10D1B000726D776172652073697A652E204F66669D
:10D1C0007365742069732030782530387820616E5B
:10D1D00064206669726D776172652073697A652073
:10D1E0006973203078253038782E00457261736578
:10D1F000206F7065726174696F6E206661696C651D
:10D2000064004372656174696E67206F626A65636A
:10D210007420776974682073697A653A2025642ED2
:10D22000204F66667365743A203078253038782C44
:10D23000204352433A203078253038780048616ED8
:10D24000646C65204E52465F4446555F4F505F4FB9
:10D25000424A4543545F57524954452028646174FB
:10D260006129005772697465207265717565737400
:10D2700020746F6F206C6F6E670048616E646C6520
:10D28000204E52465F4446555F4F505F4352435FC6
:10D2900047455420286461746129004F66667365B0
:10D2A000743A25642C204352433A3078253038783C
:10D2B0000048616E646C65204E52465F4446555F7F
:10D2C0004F505F4F424A4543545F4558454355547C
:10D2D000452028646174612900496E76616C696437
:10D2E00020646174612E2065787065637465643AAA
:10D2F0002025642C20676F743A2025640048616EF5
:10D30000646C65204E52465F4446555F4F505F4FF8
:10D31000424A4543545F53454C4543542028646179
:10D3200074612900637263203D20307825782C20B9
:10D330006F6666736574203D20307825782C206DEB
:10D3400061785F73697A65203D20307825780049DF
:10D350006E76616C6964206F626A656374207479AB
:10D36000706520696E20726571756573742E004951
:10D370006E76616C6964206F70636F64652072659E
:10D380006365697665643A20307825782E004661B9
:10D39000696C656420746F207363686564756C657F
:10D3A000206F626A65637420657865637574653A99
:10D3B00020307825782E0057686F6C65206669727A
:10D3C0006D7761726520696D61676520726563655F
:10D3D000697665642E20506F737476616C69646140
:10D3E00074696E672E00526571756573742068618B
:10D3F0006E646C696E6720636F6D706C6574652E0A
:10D4000020526573756C743A203078257800416C31
:10D410006C20666C617368206F7065726174696FEF
:10D420006E73206861766520636F6D706C657465DE
:10D43000642E2044465520636F6D706C657465647E
:10D440002E006E72665F6466755F7265715F6861FB
:10D450006E646C65720043616C6C696E67206E72FD
:10D46000665F6466755F73657474696E67735F6920
:10D470006E697428292E2E2E006E72665F646675A2
:10D480005F666C6173685F696E69742829206661E4
:10D49000696C65642077697468206572726F723A8E
:10D4A00020257800526573746F72696E672073650A
:10D4B0007474696E67732066726F6D206261636B4E
:10D4C00075702073696E6365207468652061707083
:10D4D000206861732074616D70657265642077697E
:10D4E000746820746865206F66662D6C696D697458
:10D4F000207061727473206F662074686520736594
:10D500007474696E677320706167652E007365744B
:10D5100074696E67735F7772697465282920666124
:10D52000696C65642077697468206572726F723AFD
:10D5300020257800526573746F72696E6720736579
:10D540007474696E67732066726F6D206261636BBD
:10D5500075702073696E63652074686520736574E7
:10D5600074696E6773207061676520636F6E7465A0
:10D570006E74732061726520696E76616C696420D7
:10D5800028435243206572726F72292E00526573D0
:10D59000657474696E6720626F6F746C6F61646527
:10D5A000722073657474696E67732073696E636546
:10D5B000206E65697468657220746865207365748F
:10D5C00074696E67732070616765206E6F72207476
:10D5D0006865206261636B75702061726520766199
:10D5E0006C69642028435243206572726F72292E41
:10D5F0000053657474696E6773204F4B004261631A
:10D600006B696E672075702073657474696E6773DB
:10D61000207061676520746F206164647265737344
:10D6200020307825782E00433A2F6E5246355F53CE
:10D63000444B5F31352E322E302F636F6D706F6E1D
:10D64000656E74732F6C69627261726965732F62A3
:10D650006F6F746C6F616465722F6466752F6E7284
:10D66000665F6466755F73657474696E67732E6355
:10D6700000436F756C64206E6F7420706572666F06
:10D68000726D206261636B7570206F6620626F6FD0
:10D69000746C6F616465722073657474696E67730E
:10D6A00021204572726F723A2030782578004465E7
:10D6B0007374696E6174696F6E2073657474696EDA
:10D6C000677320617265206964656E746963616C5B
:10D6D00020746F20736F757263652C207772697484
:10D6E00065206E6F74206E65656465642E20536BD3
:10D6F000697070696E672E0057726974696E672071
:10D7000073657474696E67732E2E2E004572617393
:10D71000696E67206F6C642073657474696E6773DB
:10D720002061743A2030782530387800436F756C6A
:10D7300064206E6F74206572617365207468652063
:10D7400073657474696E6773207061676521004347
:10D750006F756C64206E6F742077726974652074C5
:10D760006865204446552073657474696E6773203C
:10D770007061676521006E72665F6466755F7365D0
:10D780007474696E67730045726173696E672073A4
:10D79000657474696E677320706167652061646485
:10D7A0006974696F6E616C20646174612E006E72C1
:10D7B000665F6466755F73657474696E67735F73C3
:10D7C000766369005368757474696E6720646F7757
:10D7D0006E207472616E73706F7274732028666F3E
:10D7E000756E643A20256429004661696C65642081
:10D7F000746F2073687574646F776E207472616ED5
:10D8000073706F72742025642C206572726F7220A1
:10D81000256400496E697469616C697A696E672074
:10D820007472616E73706F7274732028666F756E98
:10D83000643A20256429004661696C656420746F30
:10D8400020696E697469616C697A65207472616EB1
:10D8500073706F72742025642C206572726F722051
:10D86000256400456E746572206E72665F6466752D
:10D870005F6170705F69735F76616C6964004E6FA1
:10D880002076616C69642061707020746F20626F13
:10D890006F742E0043524320636865636B206F668C
:10D8A00020617070206661696C65642E2052657419
:10D8B00075726E2025640052657475726E207472E4
:10D8C00075652E20417070207761732076616C69D8
:10D8D0006400456E746572206E72665F6466755F83
:10D8E00063616368655F70726570617265282900A5
:10D8F00072657175697265645F73697A653A203023
:10D900007825782E00747275650066616C73650009
:10D9100073696E676C655F62616E6B3A2025732E6A
:10D92000006B6565705F6170703A2025732E006B27
:10D930006565705F736F66746465766963653A20C8
:10D9400025732E0053445F50524553454E543A20A0
:10D9500025732E0042616E6B20636F6E74656E746A
:10D96000733A0042616E6B203020636F64653A2029
:10D970003078253032783A2053697A653A20307809
:10D9800025780042616E6B203120636F64653A2018
:10D990003078253032783A2053697A653A203078E9
:10D9A000257800433A2F6E5246355F53444B5F3122
:10D9B000352E322E302F636F6D706F6E656E7473FF
:10D9C0002F6C69627261726965732F626F6F746C1C
:10D9D0006F616465722F6466752F6E72665F646630
:10D9E000755F7574696C732E6300706173733A2090
:10D9F00025642E0063616368655F616464726573AA
:10DA0000733A20307825782E0063616368655F740F
:10DA10006F6F5F736D616C6C3A2025732E006B65C0
:10DA200065705F6669726D776172653A2025732E45
:10DA30000064656C6574655F6D6F72653A2025736F
:10DA40002E0041626F7274696E672E2043616E6EA4
:10DA50006F7420666974206E6577206669726D77D1
:10DA6000617265206F6E2064657669636500496E3A
:10DA700076616C69646174696E67206170702E00F4
:10DA8000433A2F6E5246355F53444B5F31352E3249
:10DA90002E302F636F6D706F6E656E74732F6C69AF
:10DAA000627261726965732F626F6F746C6F61640B
:10DAB00065722F6466752F6E72665F6466755F7639
:10DAC000616C69646174696F6E2E6300496E69747C
:10DAD00020636F6D6D616E64206C6172676572208A
:10DAE0007468616E2065787065637465642E0045A6
:10DAF0007865637574652077697468206661756CF4
:10DB00007479206F6666736574005369676E61741B
:10DB10007572652072657175697265642E2043683F
:10DB200065636B696E67207369676E617475726592
:10DB30002E004E6F207369676E6174757265206682
:10DB40006F756E642E00496E76616C69642073692E
:10DB5000676E617475726520747970650043616CDD
:10DB600063756C6174696E6720696E697420706199
:10DB7000636B657420686173682028696E6974201E
:10DB80007061636B6574206C656E3A2025642900B2
:10DB9000566572696679207369676E61747572651E
:10DBA000005369676E6174757265206661696C65A2
:10DBB0006420286572725F636F64653A203078254F
:10DBC0007829005369676E61747572653A0048611F
:10DBD00073683A005075626C6963204B65793A004E
:10DBE000496D6167652076657269666965640042A2
:10DBF0004C2073697A652028256429206F76657228
:10DC0000206C696D6974202825642900496E697447
:10DC1000207061636B657420646F6573206E6F7430
:10DC200020636F6E7461696E2076616C6964206632
:10DC300069726D776172652073697A650043616E00
:10DC400027742066696E6420726F6F6D20666F7234
:10DC50002075706461746500577269746520616431
:10DC600064726573732073657420746F2030782537
:10DC7000303878004661696C656420746F20646593
:10DC8000636F646520696E6974207061636B65748D
:10DC9000006D616A6F72006D696E6F72004861732A
:10DCA0006820766572696669636174696F6E2E209B
:10DCB0004669726D77617265207374617274206158
:10DCC0006464726573733A20307825782C20736908
:10DCD0007A653A203078257800436F756C64206E41
:10DCE0006F742072756E2068617368207665726942
:10DCF0006669636174696F6E20286572725F636F15
:10DD000064652030782578292E0048617368207674
:10DD10006572696669636174696F6E206661696CBA
:10DD200065642E00457870656374656420465720ED
:10DD3000686173683A0041637475616C20465720CE
:10DD4000686173683A00496E76616C6964617469F0
:10DD50006E67206F6C64206170706C6963617469B8
:10DD60006F6E20696E2062616E6B20302E005468E9
:10DD70006520536F667444657669636520646F65DA
:10DD800073206E6F7420636F6E7461696E207468A7
:10DD900065206D61676963206E756D6265722069CB
:10DDA00064656E74696679696E6720697420617351
:10DDB000206120536F66744465766963652E005454
:10DDC000686520536F66744465766963652073697E
:10DDD0007A6520696E2074686520696E666F2073AD
:10DDE000747275637420697320746F6F20736D6132
:10DDF0006C6C20636F6D7061726564207769746804
:10DE0000207468652073697A65207265706F72741A
:10DE1000656420696E2074686520696E697420638A
:10DE20006F6D6D616E642E00536F66744465766924
:10DE300063652075706461746520697320612025B5
:10DE4000732076657273696F6E2075706461746596
:10DE50002E2043757272656E743A2025642E204E12
:10DE600065773A2025642E00496E76616C6964619D
:10DE700074696E6720617070206265636175736597
:10DE800020697420697320696E636F6D70617469B5
:10DE9000626C6520776974682074686520536F66CA
:10DEA000744465766963652E004D616A6F72205314
:10DEB000442075706461746520627574206E6F20F3
:10DEC000424C2E2041626F727420746F2061766F15
:10DED000696420696E636170616369746174696EFD
:10DEE000672074686520424C2E0050423A20496EEB
:10DEF0006974207061636B65742064617461206C67
:10DF0000656E3A2025640048616E646C65723A2043
:10DF1000496E76616C69642070726F746F636F6CA8
:10DF200020627566666572206D5F70625F737472E1
:10DF300065616D006E72665F6466755F76616C69BF
:10DF4000646174696F6E00433A2F6E5246355F53B9
:10DF5000444B5F31352E322E302F636F6D706F6EF4
:10DF6000656E74732F6C69627261726965732F627A
:10DF70006F6F746C6F616465722F6466752F6E725B
:10DF8000665F6466755F7665725F76616C69646111
:10DF900074696F6E2E6300496E76616C69642066E9
:10DFA00069726D7761726520747970652E00496EB3
:10DFB00076616C6964206861736820747970652E7D
:10DFC000004E6F2048572076657273696F6E2E0081
:10DFD0004661756C74792048572076657273696F55
:10DFE0006E2E00534420726571206E6F74206D6533
:10DFF000742E0046572076657273696F6E20746FB9
:10E000006F206C6F772E0046572076657273696FAC
:10E010006E206D697373696E672E006E72665F6441
:10E0200066755F7665725F76616C69646174696F4D
:10E030006E00010000070000E4B10700ECB107002A
:10E0400008000000D4B10700E4B107000800000098
:10E05000ECB10700F4B10700080000006E72665FC3
:10E060007364680073645F626C655F6366675F73A7
:10E07000657428292072657475726E656420257335
:10E08000207768656E20617474656D7074696E6761
:10E0900020746F2073657420424C455F434F4E4E91
:10E0A0005F4346475F4741502E0073645F626C6573
:10E0B0005F6366675F736574282920726574757283
:10E0C0006E6564202573207768656E2061747465C1
:10E0D0006D7074696E6720746F2073657420424C94
:10E0E000455F4741505F4346475F524F4C455F4352
:10E0F0004F554E542E0073645F626C655F636667B4
:10E100005F73657428292072657475726E6564206A
:10E110002573207768656E20617474656D7074690D
:10E120006E6720746F2073657420424C455F434FC7
:10E130004E4E5F4346475F474154542E0073645F21
:10E14000626C655F6366675F73657428292072651A
:10E150007475726E6564202573207768656E206122
:10E160007474656D7074696E6720746F2073657464
:10E1700020424C455F434F4D4D4F4E5F4346475FF6
:10E1800056535F555549442E0073645F626C655F5A
:10E190006366675F73657428292072657475726E93
:10E1A0006564202573207768656E20617474656DE1
:10E1B0007074696E6720746F2073657420424C45DB
:10E1C0005F47415454535F4346475F415454525F45
:10E1D0005441425F53495A452E0073645F626C6537
:10E1E0005F6366675F736574282920726574757252
:10E1F0006E6564202573207768656E206174746590
:10E200006D7074696E6720746F2073657420424C62
:10E21000455F47415454535F4346475F5345525609
:10E220004943455F4348414E4745442E00496E737C
:10E23000756666696369656E742052414D20616C34
:10E240006C6F636174656420666F7220746865200A
:10E25000536F66744465766963652E004368616E2A
:10E260006765207468652052414D20737461727433
:10E27000206C6F636174696F6E2066726F6D203001
:10E2800078257820746F20307825782E004D6178BD
:10E29000696D756D2052414D2073697A6520666FF6
:10E2A00072206170706C69636174696F6E2069734C
:10E2B00020307825782E0073645F626C655F656E30
:10E2C00061626C6528292072657475726E656420C0
:10E2D00025732E00BCB10700C4B107000800000080
:10E2E0006E72665F7364685F626C6500F4B107000C
:10E2F000FCB10700080000006E72665F7364685F1F
:10E30000736F6300202020202020202020682828F0
:10E3100028282020202020202020202020202020ED
:10E320002020202048101010101010101010101075
:10E330001010101084848484848484848484101055
:10E340001010101010818181818181010101010172
:10E35000010101010101010101010101010101109E
:10E360001010101010828282828282020202020247
:10E37000020202020202020202020202020202106F
:10E380001010102000070320041702010857104046
:10E390008000000038E50700FCE3070010E50700F7
:10E3A00053756E004D6F6E005475650057656400BF
:10E3B00054687500467269005361740000000000E3
:10E3C0004A616E00466562004D61720041707200E4
:10E3D0004D6179004A756E004A756C0041756700A1
:10E3E000536570004F6374004E6F760044656300A0
:10E3F00000000000414D00504D00000034E50700D2
:10E4000030E5070030E5070030E5070030E507009C
:10E4100030E5070030E5070030E5070030E507008C
:10E4200030E50700FFFFFFFFFFFFFFFFFFFFFFFFDC
:10E43000FFFF000070E40700A0E30700ACE4070062
:10E44000C0E30700F4E3070054E4070004E5070015
:10E4500060E40700256D2F25642F2579000000005A
:10E46000256120256220256520255420255900009E
:10E4700053756E646179004D6F6E646179005475F7
:10E480006573646179005765646E657364617900D2
:10E4900054687572736461790046726964617900C9
:10E4A0005361747572646179000000004A616E7591
:10E4B000617279004665627275617279004D6172B0
:10E4C000636800417072696C004D6179004A756E35
:10E4D00065004A756C790041756775737400536502
:10E4E0007074656D626572004F63746F626572006F
:10E4F0004E6F76656D62657200446563656D626539
:10E500007200000025483A254D3A255300000000CE
:10E510008DAE0700A9AE0700B5AE0700C1AE07007B
:10E52000DDAE0700E9AE0700F5AE070003AF070058
:10E53000000000002E00000043000000504F53492F
:04E54000580000007F
:10E5440000000000FF0000000000000000000000C8
:10E5540000000000000000000000000000000000B7
:10E5640000000000010000000C2000201C200020FE
:10E574000090D003FF00FFFF0100000000E007004F
:10E5840094E3070094E3070094E3070094E307008F
:04E5940094E3070005
:020000020000FC
:020000041000EA
:0410140000300700A1
:0410180000E00700ED
:0400000370003379DD
:00000001FF
